:1000000006C500000C94B9313AC5000038C500009F
:1000100036C5000034C5000032C5000030C5000000
:100020002EC500002CC500000C94EF2F0C94D73087
:100030000C94A42F24C5000022C5000020C5000098
:100040001EC500001CC500001AC5000018C5000030
:1000500016C500000C94CB2F12C5000010C500007F
:100060000EC500000CC500000AC5000008C5000050
:1000700006C5000004C5000002C5000000C5000060
:10008000FEC40000FCC40000FAC40000F8C4000074
:10009000F6C40000F4C40000F2C40000F0C4000084
:1000A000EEC40000ECC40000EAC4000005010980B1
:1000B000A101850319012AB700150126B700950192
:1000C00075108100C0050C0901A101850419012AE0
:1000D000A002150126A002950175108100C00660DE
:1000E000FF0961A1010962150026FF00952075082E
:1000F00081020963150026FF00952075089102C052
:1001000005010906A101050719E029E715002501E8
:10011000950875018102950175088101050719008F
:1001200029FF150026FF00950675088100050819AE
:1001300001290515002501950575019102950175A7
:10014000039101C00000000000000000000000005A
:10015000000000000000000000000000000000009F
:1001600000000000000000007E0F00D4FFFFFFC76A
:100170000000007800000000000000002A2B28008A
:100180000000000000000000000000000000002946
:10019000000000002C1E3420212224342627252E86
:1001A000362D3738271E1F202122232425263333BE
:1001B000362E37381F0405060708090A0B0C0D0EEA
:1001C0000F101112131415161718191A1B1C1D2FB6
:1001D0003130232D350405060708090A0B0C0D0ED6
:1001E0000F101112131415161718191A1B1C1D2F96
:1001F0003130354C09025B00030100A0FA0904000C
:10020000000103010100092111010001224400073E
:100210000581030800010904010002030000000930
:10022000211101000122220007058203200001079D
:100230000503032000010904020001030000000976
:100240002111010001223200070584032000011260
:100250000100020000000810CB5733100301020315
:10026000011C037600690061006C003A00660036EC
:10027000003400630032006200330063000000229B
:10028000035100750065006600720065006E006332
:1002900000790020005200650076002E0020003317
:1002A0000000000E034B0065006500620069006FEE
:1002B000000000040309043A003B00167C1E001FE6
:1002C0000020002100220023003C003D002B0014F0
:1002D000001A0008001500170000003E003F00391A
:1002E0000004001600070009000A00000040004159
:1002F00000E10000001D001B00060019000500427F
:10030000004300E000E200E300215200002C000066
:100310000024002500260027002D002E004C002A76
:10032000004A001C0018000C00120013002F0030BF
:100330000031004D000B000D000E000F00330034A3
:1003400000000028004B0011001000360037003874
:10035000000000E50052004E0021522C00E600E4AF
:1003600000E7000000500051004F0001000100169E
:100370007C3A003B003C003D003E003F0001000194
:1003800000207821780100520001000100000001E6
:1003900000010001000100500051004F0001000069
:1003A0000001000100010000000100010001000146
:1003B0000001000100010035020100010001000000
:1003C000000100000040004100420043004400459D
:1003D000004C002A000100010001000100010001A1
:1003E0000001000100010001000100010001000105
:1003F00000010001000000010001000100010001F6
:1004000000010001000000010001000100010001E5
:10041000000100010001000000010001000100AA2C
:1004200000A9004E004B0022782178AC00AB0022DE
:1004300023252628292A2C2D2F3032333536383AD9
:100440003B3D3E4042434547494A4C4E505153552F
:1004500057595A5C5E6062646668696B6D6F717350
:100460007577797B7D7F81838587898A8C8E909251
:100470009496989A9C9E9FA1A3A5A7A8AAACAEAF5C
:10048000B1B3B4B6B8B9BBBCBEBFC1C2C3C5C6C7A1
:10049000C9CACBCCCDCED0D1D2D2D3D4D5D6D7D752
:1004A000D8D9D9DADADBDBDBDCDCDCDCDCDDDDDD9A
:1004B000DDDCDCDCDCDCDBDBDBDADAD9D9D8D7D796
:1004C000D6D5D4D3D2D2D1D0CECDCCCBCAC9C7C643
:1004D000C5C3C2C1BFBEBCBBB9B8B6B4B3B1AFAE81
:1004E000ACAAA8A7A5A3A19F9E9C9A989694929027
:1004F0008E8C8A89878583817F7D7B7977757371FF
:100500006F6D6B6968666462605E5C5A59575553DB
:1005100051504E4C4A4947454342403E3D3B3A3894
:1005200036353332302F2D2C2A292826252322FF39
:10053000AA7F55400102030C0D0E0F0007060504AB
:100540000B0A090800010101010101010101020278
:100550000202020202020203030303030303030471
:10056000040404040404050505050506060606063C
:10057000070707070708080808090909090A0A0AF6
:100580000B0B0B0C0C0C0D0D0D0E0E0E0F0F0F1098
:100590001011111112121313141415151616171722
:1005A000181819191A1A1B1B1C1D1D1E1E1F20208E
:1005B000212222232424252626272829292A2B2CD8
:1005C0002D2D2E2F30313232333435363738393AFB
:1005D0003B3C3D3E3F404142434445464748494AF3
:1005E0004C4D4E4F50515354555658595A5B5D5EC1
:1005F0005F616264656668696B6C6D6F707273755C
:1006000077787A7B7D7E8082838587888A8C8E8FBF
:1006100091939596989A9C9EA0A2A3A5A7A9ABADED
:10062000AFB1B3B5B7BABCBEC0C2C4C6C9CBCDCFDB
:10063000D1D4D6D8DBDDDFE2E4E7E9EBEEF0F3F589
:10064000F8FAFDFF1E0F0500047F3F1F643214649B
:100650003214783C1E1E140A05FD377A585A0000E1
:1006600004E6D6B4460200210116000000742FE50E
:10067000A3E00E9003495D003D8889C65436C31738
:100680004FE4E5014D6F8DD6A60C93036C2ABA3268
:100690000B67C912CA2E4BF24146C9FCB1ED076483
:1006A000B2AB47408C484DCE0637AD2D1B90B946B6
:1006B0004D525FFB23D34389C0DCF63AA8FAF874A5
:1006C000DF80ECE1E16FEABDFA1FD5CF95BC9EB5A6
:1006D000C820CDA25FF86E05A0F4416652E804661A
:1006E00017865A9C94237B5C7A4F152BF5F06F4547
:1006F000FEE103814C9039EC5D2CA80FBF50EC2932
:10070000E032E126670F2851806289E2BA835926D8
:10071000941BE65A616886CF417FFF3BC3A1C37239
:100720004BFB8747F73E083EAF42D560AD79FDEB06
:100730002095CD6992E50A759BC554D098C8721F63
:10074000F4C6200836E587C66643A104C5351ED722
:1007500072B5C9A24B621C308E0C28B96F865C4DF5
:10076000FF8FD5213E02077ADFFC7D162214F04B65
:10077000892D335BC9560A11D251EF6DCD282879E6
:10078000EC9D5D088B73ABDCC58168E41001C991F9
:100790006FFD2D80AB2669E379FA3B839B390F8887
:1007A00083C5268005288E5E0C155CC6F217DF9384
:1007B000B4973A0BCAC545AC69045DA9F68C40F7FD
:1007C000116D6E4D19A13D72ACFB73E2BC98F349FB
:1007D0003340A2F1252EA956CEB50D2F15C1C26A00
:1007E00005E20571B3CC3D6D2012CE8DA7945A1D44
:1007F0001FA29466B297A7C6E44D7FE61F63970ECB
:1008000044470C95E40012BCA3D31D44AF4C20EF29
:10081000978DBA3F3DF0669086950B24C2A785520E
:10082000C1830A6C80550726F8AC81BF6A42012556
:10083000249CA838409682A3A80E39A5F39081C1C4
:10084000E38DA7B0448CBA41536EBD9D19952FF826
:10085000E70E38640DAEC9A7B73335A99FA7176C4B
:10086000D46B5F02FCD483638F42D5E0B5B6A09809
:10087000A87F451FB0CB56A672289F369D6FA788CC
:10088000AF7B41A3A6295471332B01A51F2D7730CF
:100890003B0EF3AA8B62EE154DDE80FA8E5D277E4D
:1008A000442726CBFFF020E3CABB35B5DD22EEC8D6
:1008B0002DA993B7E33A0D0A4530E53539325ACAC6
:1008C000348889DB87CBF4889D4C3A5EB4851EEE74
:1008D000D5F11661280F2E8874DB7742F521B8A474
:1008E0002911C4852C3DF2E30D406633371841973A
:1008F000C00CAA30E5B8CBE6923A9F43C111D6EEC0
:10090000613BDD7089E42EDFFC40763E044B91C0F4
:10091000015707DB3C3F86EDD1BF1B3D21AD8CD994
:100920005DC736E9107F6429AB59D1BF30FAC80BD7
:1009300030EE7BA9C36D47BBFF733A8D5C9A5DD4E3
:100940006A321769126DADC2A9AF100E70C1D9E934
:10095000A2E8D94977AAF1F81B9FF940440897A863
:10096000DD75F89457A50901DF886D7837D9623AAB
:10097000BF0B3220BC4814D084E2252AA8E0BE6C0C
:1009800043D2D2D7CA652CE3A89942E8739A4EB2F3
:10099000A8489B1DEAD80961BE7840720E2637A888
:1009A000A8BFE955BF55DC46A1DB133E3242463AAB
:1009B00020446CDE3A7E604EEE1F35D6B5AA2B97EA
:1009C0008A000000005A7451E6F3D4AFE10001E55B
:1009D00006911D0000AE1D9E1BB1C467FB02000006
:1009E000000004595A504F52514A4D4B4E2A4C2F39
:1009F00030B6B7ABACBBBCA9AABDBE0D0E0B0F1A6F
:100A00000508050905071811130408120C00112424
:100A10001FBECFEFDAE0DEBFCDBF04B603FE18C0C5
:100A20008091A1049091A204A091A304B091A40488
:100A30008730904BA740B04B59F41092A10410920C
:100A4000A2041092A3041092A404E0E0F8E3099534
:100A500024E0A2E4B2E001C01D92A13AB207E1F79E
:100A600012E0A0E0B1E0E8E2FAE602C005900D92E3
:100A7000A234B107D9F70E94D0270C94DC34C0CA45
:100A80009C01FB019A9581159F4120F5832F817070
:100A9000B32FB270AA27732F74706627532F587024
:100AA000442734FF0DC08295807FAB2B09F0806214
:100AB000672B09F08064452B09F08068099508953B
:100AC000AB2B09F08260672B09F08460452BB1F3F2
:100AD0008860F4CF80E0F2CF0C9438330895982FDB
:100AE00092959F7024E0911102C020E0982F892FE9
:100AF00086958695811511F02E5F982F892F869502
:100B0000820F089590916F01911529F081FD02C027
:100B10002E9A08952E980895809344040895809302
:100B20004504089521E030E001C0220F8A95EAF7DC
:100B300080914504822BF3CF21E030E0A90102C06F
:100B4000440F551F8A95E2F7CA018095909145049C
:100B50008923E5CF9B01677091E001C0990F6A95E9
:100B6000EAF763E0369527956A95E1F7B901660FD4
:100B7000771F260F371FFA01E20FF31F40E050E006
:100B8000682F70E08191DF019B01042E02C0369531
:100B900027950A94E2F721702195282729232827F1
:100BA0002E934F5F5F4F4330510561F708959C01CD
:100BB000A82FA77083E0369527958A95E1F7C9019C
:100BC000880F991F820F931FFB01E80FF91F40E068
:100BD00050E080E0219130E00A2E02C03695279542
:100BE0000A94E2F721703327042E01C0220F0A94E1
:100BF000EAF7822B4F5F5F4F4330510559F7089555
:100C0000282F862F903F71F09A3068F4293050F4E5
:100C1000622F70E029E0929F600D711D11244DEA52
:100C200053E098CF08959C5F9230E0F7622F70E018
:100C30004AEA53E0F6CF903FB9F09A3070F4893029
:100C400098F4282F30E06DEA73E0A901E9E09E9F57
:100C5000400D511D1124CA01AACF9C5F923020F48F
:100C60006AEA73E090E0F8CF80E00895909145043F
:100C700021E030E0F90101C0EE0F8A95EAF7D901D1
:100C800002C0AA0FBB1F6A95E2F7EA2B01C0220F30
:100C90004A95EAF7892F8E23E81303C0892F822B08
:100CA0003ECF2095822F8923FBCF80914D049091D8
:100CB0004C04981301C008958F5F8770FACF90910C
:100CC00047048095892380934704282F277021119A
:100CD00010C0891771F09091A00492FF0AC0869508
:100CE0008695869529DF1092470410924904109248
:100CF00048040895982F9095809142048923809309
:100D00004204089580914104811531F0109241040C
:100D100010924B0410924A04089590919F0492FF00
:100D200010C041E0282F2471243009F040E031E068
:100D3000282F2871283009F030E0431711F02CE0FB
:100D4000822793FF10C041E0282F2471243109F03D
:100D500040E031E0282F2871283109F030E04317B6
:100D600011F02CE082273091A00430FF10C051E038
:100D7000282F2171213009F050E041E0282F2871FF
:100D8000283009F040E0541711F029E0822731FFA4
:100D900010C041E0282F2171213109F040E031E0FD
:100DA000282F2871283109F030E0431711F029E08D
:100DB000822794FD877E0895CF93DF93EC01811500
:100DC00022E5920708F046C0811540E5940708F037
:100DD000C1C0803E910520F58D3C910508F095C07D
:100DE000883A910570F4853A910508F08BC08130FE
:100DF000910561F10497813A910540F1C0E0D0E09E
:100E000025C0885A91094B97C8F7C85AD0E0CC0F33
:100E1000DD1FCB52DE4F0990D881C02DD46416C09F
:100E20008115904488F4C11580E2D80708F0A8C065
:100E3000C83ED10558F0CE019A9581159F41F0F634
:100E40008D2F6BDFD82F02C0DF70D06ACE01DF910B
:100E5000CF910895803842E59407C8F5803652E571
:100E6000950708F05BC0C03482E5D807D0F4C032E3
:100E700092E5D90708F04BC08C2F8695869520E225
:100E8000829FC0011124C37021E030E0A90102C09B
:100E9000440F551FCA95E2F7EA01C82BD92BDD682C
:100EA000D5CF8C2F86958695877050E2859FC0019F
:100EB0001124C37021E030E0A90102C0440F551F86
:100EC000CA95E2F7EA01C82BD92BDC68BFCF803C7A
:100ED00052E5950758F48F71C03AD245A0F590E0DD
:100EE000982F8827EC01C46FD06AB0CF805C924500
:100EF000809708F083CFDC2FCC27CC27DF71C06F21
:100F0000D06AA4CFA497D064A1CFD0659FCFCF7172
:100F1000D0E0DC2FCC27C16FD06A98CF869586951C
:100F2000877020E2829FC0011124C37021E030E06D
:100F3000A90102C0440F551FCA95E2F7EA01C82B68
:100F4000D92BDA6883CFE9DEC82FD0E0DC2FCC279D
:100F5000D0627CCF8F71E1DE93E0CC0FDD1F9A95DC
:100F6000E1F7CC27DF70282F30E084FF05C050E187
:100F7000859F900111243327C22BD32BD06966CFD4
:100F80008D2F8F71CADED82FE3CF80E00895F894BB
:100F9000E82FE295EF70F0E041A18F7021E030E0A2
:100FA000B90102C0660F771F8A95E2F7CB01962F31
:100FB0009095942391A392A1892B82A3789408956C
:100FC00081E080935D0308950895CF92DF92EF92C0
:100FD000FF921F93CF93DF93172FE82FF0E0EC5B86
:100FE000FA4F71110CC0E4918E2F7E2F6E2FDF917E
:100FF000CF911F91FF90EF90DF90CF900895E62E54
:10100000F12CC72ED12CF491EF2F86E0689F900130
:101010001124CFEFD0E0C901BE010E940B33AB0118
:10102000EE0CFF1C65E5649FC001659F900D1124C7
:10103000E81AF90A6E2D660F6E0D7E01EC18FD0898
:10104000FE9DD001FF9DB00D11248B2F169F7001C6
:101050001124EF2CFF246E01CE18DF087601FE9DCF
:101060006001FF9DD00C11247E01E61AF108B70142
:10107000169F7001179FF00C1124EF2CFF24CE193E
:10108000DF09FC9F7001FD9FF00C11247F2D433080
:101090005105C1F02C3F334058F441305105B1F0B7
:1010A0004230510509F0A2CFEB2F8F2D7F2F9ECF1D
:1010B0004430510571F04630510509F497CF7B2F2C
:1010C0008D2D94CF7D2DEB2F8F2F90CF7F2FED2D5A
:1010D0008DCFEF2D7B2FF8CFCF93DF93982F762FE7
:1010E000842FE901692F71DF472F282FFE01FF2789
:1010F000EC5CFA4FE49180911601E81B8E2F90E092
:1011000038D3DF91CF91089580913804843028F44A
:10111000837084608093380408958C3AE8F3837078
:10112000886AF8CFCF938091380480FF03C0D9D567
:10113000CF910895C091180180911901C817B8F78F
:10114000EC2FF0E0EC5CFA4FE49180911601E81B83
:1011500020E040E060E08E2F90E00BD3CF5FECCF3B
:101160000F931F93CF93DF93D82F162F042F8091C7
:101170003804C091180180FD14C0DF91CF911F91F8
:101180000F910895EC2FF0E0EC5CFA4FE491809120
:101190001601E81B202F412F6D2F8E2F90E0E9D2F2
:1011A000CF5F80911901C81768F3BCDFE6CFCF93FA
:1011B000DF93EC0120913B049C81892F817090FD8D
:1011C000822F692F627091FD622F492F447092FD2A
:1011D000422FC6DF8C8190E00196877099278C831F
:1011E000DF91CF910895982F762F842F2091380486
:1011F00020FF07C0692FE9DE962F672F482F892F20
:10120000AFCF0895CF93DF93EC01E8E3F4E043819F
:1012100062818C81E8DF8C818F5F8C83DF91CF913D
:101220000895E5E3F4E01182828184608283089569
:10123000E8E3F4E080818E7F8083F3DFE5E3F4E090
:101240008281816082836ECFCF93DF93EC01EC814A
:10125000F0E0E15DFB4F4491E8E3F4E062818181DD
:10126000C2DF8C818F5F8C83DF91CF910895EF92E5
:10127000FF921F93CF93DF93EC0110E0EE24EA94EA
:10128000F12C60911A01161768F04CDF8C819A815D
:1012900090FF1DC08F5F8C83DF91CF911F91FF90D6
:1012A000EF90089520911801210F3327331F70E02C
:1012B000C7010E941F33962F8C8140913B0460919F
:1012C0003A04199F800D112407DF1F5FDACF815088
:1012D000E2CFA0E0B0E0EFE6F9E00C94D132EC010F
:1012E0008A8101E080FD0FEF8C81811109C00130FE
:1012F00019F480911A0181508093F30281E08C836C
:1013000010E080911A011817B0F00CDF9091F302F1
:10131000013009F053C080911A018150911519F0E4
:101320008FEF890F91E08093F3029C83CDB7DEB7F6
:10133000E9E00C94ED32E0911801E10FF0E0EC5C93
:10134000FA4FE49180911601E81B20E040E060E054
:101350008E2F90E00ED294E0E92EF12CB12CC12E0C
:10136000D12C8091F3028B0D813114F18F70082EF6
:10137000001C00088C150D04A1F480911801960141
:10138000280F311D40913B046E2D6403A0011124F0
:10139000559547955595479560913A048091390444
:1013A0009BDEB00E81E0E81AF108D9F61F5FA9CFE5
:1013B00087FFDDCF90911A01890FD9CF892F90E057
:1013C000019660911A0170E00E941F33982FABCFF5
:1013D0001F93CF93DF93EC018C81811109C081E0D1
:1013E0008C831092F20292E09093060180930501A3
:1013F0001091180180911901181740F110E06091C7
:101400001A01161798F18EDE809105019091F20273
:10141000980F9093F20220910601280F2093060165
:10142000121654F420911A012150330B092E001C7E
:1014300000089217030634F08195809305018130EE
:1014400009F41C82DF91CF911F910895E12FF0E004
:10145000EC5CFA4FE49180911601E81B20E040E03B
:1014600060E08E2F90E085D11F5FC4CFE12FF0E0C8
:1014700070E0CF010E941F3320911801280F809146
:10148000F20230E0082E001C0008E817F0058CF08E
:1014900080910601082E001C00088E170F064CF0E4
:1014A00040913B0460913A048091390415DE1F5F3E
:1014B000A6CFF901EC5CFA4FE49180911601E81B8C
:1014C00020E040E060E08E2F90E053D1F0CFA6E026
:1014D000B0E0EDE6FAE00C94D2328D839E83AD81CC
:1014E000BE811496FC912F2F30E0D9010E94CD349B
:1014F0009B01AC010E949B346B017C0180E290E077
:101500009C012F1B3109F901A5E5B0E0A701960167
:101510000E949B3469837A838B839C839F01DF01C4
:101520000E944F339B010E9455339B01AC012C0D4F
:101530003D1D4E1D5F1D69817A818B819C810E94BA
:10154000AB34022F30E00A3240F5A901440F551F99
:10155000420F531F55954795142F1095F12C85E593
:10156000E82EE01A80911A01F81628F1DBDDAD8132
:10157000BE8114969C9181E0911519F0903219F476
:101580008FEF8093040180910401890FED81FE812A
:1015900084832696E8E00C94EE3285E590E0821B89
:1015A000930BAC01440F551F480F591F57FFD2CF63
:1015B0004F5F5F4FCFCF8E2DF1FC802F2091180110
:1015C0002F0D3327331F412F60913A0485DDF394AB
:1015D000C9CF0F931F93CF93DF93EC0100E010E08E
:1015E00090911A010917110564F09CDD8C8190E03F
:1015F0000196817099278C83DF91CF911F910F9174
:1016000008954C81809118019801280F311D609137
:101610003A048091390496950917110544F441154F
:1016200041F040913B0458DD0F5F1F4FD9CF41156A
:10163000C1F340E0F8CFFB01811520E2920728F4C6
:10164000811541E0940738F408959C01305221152A
:10165000304348F00895392F94FF02C03295307F0F
:101660002081232B208399270895462B22FF0FC02A
:10167000982F92959F708F70892B962F92959F70BF
:101680006F70692B942F92959F704F70492B982FF4
:101690009623961309C050E04095509590E048235A
:1016A000592381E0452B09F080E0089590912D03A6
:1016B000292F30E070912E03A9014F5F5F4F4370D7
:1016C00055277417150689F0255D3C4F60FB87F997
:1016D000F90184839F5F937090932D0380912B0376
:1016E0008F5F80932B0381E0089580E0089590E060
:1016F0006115E9F0855E9E4FFC0180818F3FB1F05E
:10170000E82FE295EF70F0E041A18F7021E030E02A
:10171000B90102C0660F771F8A95E2F7CB01962FB9
:101720009095942391A392A1892B82A30895845E1E
:101730009E4FE2CF90E06115A9F0855E9E4FFC01BF
:1017400020812F3F91F0E22FE295EF70E05EF0E014
:10175000808190E02F7002C0959587952A95E2F7D9
:1017600081700895845E9E4FEACF80E008956E9A5E
:101770000895FC01EE0FFF1FE80FF91FEE58FD4F13
:101780006183408322830895FC01680F791F8FEFE6
:1017900041E39191892728E030E0982F990F87FF46
:1017A00009C0892F842721503040B9F7E617F70781
:1017B00081F70895892FF7CF0F931F93CF9301E0FF
:1017C00010E0082E01C0000F0A94EAF7C09140040F
:1017D0009C2F9023911115C0909147049695969552
:1017E0009695891306C010924704109249041092EE
:1017F000480498D9C027C0934004CF911F910F91FE
:1018000008959AD9F7CF9091260489029001112466
:1018100037FF03C08093260408952F3731051CF449
:10182000980F9093260408959C0180E090E0F901C0
:10183000E80FF91FE491E41307C091E08927F9014B
:10184000E80FF11D849108950196861780F380E0DA
:10185000089580919803811569F0E091A003F091BB
:10186000A103309739F00190F081E02D309711F00D
:101870000995089580E00895A3E0B0E0E2E4FCE07B
:101880000C94D8329C018091700290917102821761
:101890009307B1F03093710220937002E091A0039E
:1018A000F091A103309761F00084F185E02D30972D
:1018B00039F083E089833B832A83CE010196099521
:1018C0002396E2E00C94F432A3E0B0E0EAE6FCE018
:1018D0000C94D8329C0180916E0290916F02821715
:1018E0009307B1F030936F0220936E02E091A00352
:1018F000F091A103309761F00084F185E02D3097DD
:1019000039F084E089833B832A83CE0101960995CF
:101910002396E2E00C94F4328091130108952FB7DE
:10192000F89480916A0290916B02A0916C02B09140
:101930006D022FBF0895962F2091A00422FF0EC0A4
:10194000682F660F660F660F692B60934704EAD80D
:10195000E6DF90934904809348040895E3C890918A
:101960004104292F2823211559F08095892380933C
:101970004104811531F0D3DF80934A0490934B04E6
:10198000089580E090E0F8CF2FB7F89460916A0254
:1019900070916B0280916C0290916D022FBF08953F
:1019A0000F931F9380919803811521F0EDDF1F9114
:1019B0000F910895E9DF0091940310919503209110
:1019C000960330919703600F711F821F931FEFCF13
:1019D00080919803811509F0A2CFE2DFCB01089531
:1019E00008950895FC019B0180916002909161022D
:1019F0008617970740F0672B29F48091E8008E77CF
:101A00008093E800C90140E0009741F4411106C00D
:101A10008091E80082FF2FC080E008952091540358
:101A20002115A9F12530A9F12091E80023FD2DC051
:101A30002091E80022FDECCF2091E80020FFE4CFC8
:101A40003091F3002091F200009719F02830310511
:101A500058F041E02830310509F040E02091E800DD
:101A60002E772093E800D0CF41914093F100019769
:101A70002F5F3F4FE9CF80915403811541F08530AE
:101A800041F08091E80083FFC3CF81E0089582E0B8
:101A9000089583E0089580915A0287FF13C08091D2
:101AA000E80082FF06C08091E8008B778093E80011
:101AB0000895809154038111F2CF089580915403C9
:101AC0008115D9F38091E80080FFF8CF8091E8007C
:101AD0008E77ECCF2091E4003091E50095E6A901E6
:101AE0002091EC00822F817020FF06C08091E800D9
:101AF00080FF06C080E008952091E80022FD1AC012
:101B000080915403811589F0853089F08091EB0034
:101B100085FD0FC02091E4003091E5004217530786
:101B2000F9F29A95E1F684E0089582E0089583E061
:101B3000089581E00895E8EDF0E080818E7F808354
:101B40001092E2001092DA001092E100A0EEB0E0F4
:101B50008C9181608C9380818F77808319BCA7EDF5
:101B6000B0E08C918E7F8C9380818F7E80831092E9
:101B700059020895E091A003F091A103309739F044
:101B80000284F385E02D309711F060E20995089505
:101B9000982F9093E900891771F07091EC002091D3
:101BA000ED005091F00021FD09C09F5F973089F74B
:101BB0008093E9000895762F242F50E03091EB00B8
:101BC0003E7F3093EB003091ED003D7F3093ED0090
:101BD0003091EB0031603093EB007093EC00209378
:101BE000ED005093F0002091EE0027FDDECF089528
:101BF000A0E0B0E0EEEFFDE00C94D232C8EDD0E012
:101C000088818F7E8883E7EDF0E08081816080832A
:101C100084E082BF81E08093590288818E7F88832F
:101C200002EE10E0F80110821092DA0081EEC82E68
:101C3000D12CF601108288818F7788838881806813
:101C4000888388818F7D888319BC109254031092F9
:101C5000580210920C031092570290EEE92EF12CCC
:101C6000F70180818B7F808388818160888342E057
:101C700060E080E08DDFF60180818E7F8083F80157
:101C8000808181608083808188608083F70180818A
:101C90008E7F8083888180618883CDB7DEB7E8E05E
:101CA0000C94EE32E0914D0490914C0429E0E9133C
:101CB00002C080E00895AE2FB0E02E9FF001112405
:101CC000E25BFB4F3181361306C03081381303C00D
:101CD0003581341304C0FD013196E770E8CF81E00F
:101CE00008953EB13F7B2EB120644FB7F89482E750
:101CF00092E0FC010196508168E02EB9000000C01E
:101D000057FF3EB9550F000000C000C000C03EB9EB
:101D100000C06A9591F752E0823A950751F74FBF9C
:101D20008FE594E00197F1F700C00000089581E08D
:101D30008093E00080E28093D8001092C9008FE188
:101D40009EE40197F1F700C0000087E090EBDC0112
:101D50008093A1049093A204A093A304B093A4043D
:101D600088E19CE00FB6F894A895809360000FBEC0
:101D700090936000FFCF0F931F93CF93DF938B015E
:101D8000EA0190915403943051F58093E9008FEF6C
:101D90009091E80095FD06C095ED9A95F1F7000049
:101DA0008A95B1F78091E80085FF19C093DE811113
:101DB00011C08091E80085FD06C08091E8008E7713
:101DC0008093E800F3CFF80181918F018093F100B7
:101DD000219779F78091E8008E778093E800DF9172
:101DE000CF911F910F910895792F603229F440E22D
:101DF00050E0682F82E0BFCF0895CF93DF93D82FB4
:101E0000C92F48E050E0682F792F81E0B4DF88E0E7
:101E1000ED2FFC2FA2E6B2E001900D928A95E1F73A
:101E2000DF91CF910895BC0143E050E084E0A3CF5F
:101E3000A0E0B0E0EEE1FFE00C94D032F82EE92E05
:101E4000B62EA72E8A01809156029AE0C92ED12C77
:101E50008A3018F0CC24C394D12CC1E0D0E06B2D93
:101E60007A2D8F2D9E2DF8010995811116C021968E
:101E7000CC16DD0694F0CC9FC001CD9F900D900D47
:101E8000112420E030E045E34A95F1F700002F5F90
:101E90003F4F28173907B9F7E2CFCDB7DEB7EAE0F1
:101EA0000C94EC329091A00492FB222720F9281781
:101EB00079F080FB92F99093A00460919F04709157
:101EC000A00484E090E00E94643482E00C945F06F9
:101ED00008951F93CF93DF93962F122F632F843093
:101EE000D8F49A30C8F44930B8F4C42FD0E0CC0FFD
:101EF000DD1F22E1929FC00DD11D112494EB899F1B
:101F0000C00DD11D1124CE0189960E944A34612F43
:101F1000CE018A960E944A34DF91CF911F91089595
:101F20000F931F93CF93DF93962F142F022F632FBE
:101F3000843018F5923008F528E0829FE0011124E2
:101F400034E0939FC0011124C80FD91FC750DD4F43
:101F500081E084279E01280F311D280F311DC90102
:101F60000E944A3481E090E0111102C083E090E0C9
:101F7000602F8C0F9D1F0E944A34DF91CF911F91DB
:101F80000F910895CF93DF93C0914204809146044E
:101F9000C82B809141048115F1F0C1DC20914A04E5
:101FA00030914B04821B930B8838934110F00E94B0
:101FB0008206D091410420E086E492E0FC01308169
:101FC000019631112F5F32E08C349307B9F721115C
:101FD0000E948206CD2BC093440248E050E062EAA2
:101FE00073E084E492E00E94FC33892BB9F088E02E
:101FF000E4E4F2E0A2EAB3E001900D928A95E1F701
:10200000E091A003F091A103309741F00280F381A9
:10201000E02D309719F084E492E00995DF91CF919B
:10202000089510924204E6E4F2E086E0DF011D929A
:102030008A95E9F780E090E01FDC80E090E044DCE6
:10204000109246049FCFEDDF2FEF84E39CE02150F8
:1020500080409040E1F700C0000088E19CE00FB6AE
:10206000F894A895809360000FBE90936000FFCF16
:10207000AAE2B0E0EEE3F0E10C94D7328AE592E018
:10208000FC0101962091F100208322E08236920724
:10209000B9F780915B02893009F457C0C8F48230E7
:1020A00009F4B2C0833009F482C0813081F180919B
:1020B000E80083FFE6C080915A0290915B029A305B
:1020C00008F0DFC0E92FF0E0E252FB4C0C94323311
:1020D0008A3009F489C08B3051F780915A028132DD
:1020E00031F780915E0290915F02892B01F7809118
:1020F000E800877F8093E800CEDC81E090915C026D
:10210000911101C080E0809314018BDFD0CF8091CA
:102110005A02813A61F68091E800877F8093E80057
:1021200080915E0290915F02892B59F060E080E01F
:1021300090E070E057DC8091E8008B778093E800B6
:10214000B6CF68E082E692E0F4CF80915A02813205
:1021500009F0ADCF80915E0290915F028D7F892B57
:1021600009F0A5CF8091E800877F8093E8008091F7
:10217000E80082FF17C09091F3008091F20002976F
:1021800031F48091F100813011F0863021F480919A
:10219000F100809313018091E8008B778093E80031
:1021A0007ADC85CF809154038111E1CF80CF80917B
:1021B0005A02813A09F07BCF80915E0290915F02D2
:1021C000892B09F074CF8091E800877F8093E80025
:1021D0008091E80080FFFCCF809114018093F10092
:1021E0008091E8008E77DACF80915A02813209F02F
:1021F0005ECF8091E800877F8093E8004CDC80917F
:102200005D028093120153CF80915A02813A09F006
:102210004ECF8091E800877F8093E8008091E800AE
:1022200080FFFCCF80911201D9CF803889F08238AD
:1022300041F580915E028F70873018F58093E90038
:102240008091EB0085FB882780F91092E90006C099
:1022500080910C03880F90915702892B9091E80090
:10226000977F9093E8008093F1001092F1008091A5
:10227000E8008E7723C0811116C080915C02813006
:1022800009F18091E80083FF0AC08091E800877F10
:102290008093E8008091EB0080628093EB00AA9627
:1022A000E3E00C94F332823061F780915C02811597
:1022B00081F01092E9008091E800877F8093E80028
:1022C000EADBDFCF81E0933009F080E080930C03FC
:1022D000F0CF80915E028F702FEF280F263088F6A6
:1022E0008093E9002091EB0020FFE3CF933031F49D
:1022F0008091EB0080628093EB00DBCF9091EB004C
:1023000090619093EB0021E030E0A90102C0440FFE
:10231000551F8A95E2F74093EA001092EA008091F7
:10232000EB008860E8CF8111ACCF10915C021F7781
:102330008091E3008078812B8093E3008091E80016
:10234000877F8093E800A7DB8091E80080FFFCCFC7
:102350008091E30080688093E30083E0111101C065
:1023600082E0809354038DCF8058823008F089CF6B
:1023700080915C0290915D028C3D53E0950791F550
:1023800083E08A838AE289834FB7F894DE0113964B
:1023900020E03EE051E2E32FF0E0509357008491BB
:1023A00020FF03C082958F703F5F8F708A30C0F02E
:1023B000895C90E08D939D932F5F243161F74FBF2F
:1023C0008091E800877F8093E8006AE270E0CE01A8
:1023D000019608DB8091E8008B778093E80051CF6D
:1023E000805DE7CF292F33272330310509F44EC014
:1023F00078F52130310509F488C08BE590E0E4EFF1
:10240000F1E02230310509F03CCF2091E800277F30
:102410002093E800209160023091610282179307B7
:1024200008F49C0140E02115310509F073C0411109
:1024300071C08091E80082FDCDCF80915403811559
:1024400049F2853039F28091E80083FFF2CFC2CFA4
:1024500080915E0290915F022132310509F446C0FD
:102460002232310509F00DCF8330910508F009CFF4
:10247000FC01EE0FFF1FE457FE4F0190F081E02DAD
:1024800087579E4FDC018C9190E010C09C01332750
:10249000823021F12330310568F4232BB9F4E3EBCA
:1024A000F2E0E4918E2F90E0E3EBF2E0009709F484
:1024B000E8CEABCF2330310509F0E3CEE1E6F2E020
:1024C000E4918E2F90E0E1E6F2E0F0CFE3EAF2E073
:1024D000E4918E2F90E0E3EAF2E0E8CFEFE7F2E05C
:1024E000E4918E2F90E0EFE7F2E0E0CF83309105AA
:1024F00008F0C7CEFC01EE0FFF1FEE56FE4F019015
:10250000F081E02D89E090E080CF82E190E0EFE47F
:10251000F2E07BCF80915403811509F45BCF8530C5
:1025200009F458CF8091E80083FD54CF8091E800F2
:1025300082FD7FCF8091E80080FF75CF9091F300FE
:102540008091F2002115310519F08830910550F085
:1025500041E0089709F040E08091E8008E77809391
:10256000E80061CF44914093F10031962150310948
:102570000196E8CF803809F084CE8091E800877F0B
:102580008093E800809158028093F10070CE811111
:1025900078CE10915C02123008F073CE8091E80082
:1025A000877F8093E8001093580275DA1115D9F0EF
:1025B00084E08093540342E061EC81E0E9DA42E296
:1025C00061EC84E0E5DA42E261EC82E0E1DA42E2E9
:1025D00060EC83E0DDDA80915403843051F482E0D2
:1025E000809315014ECE8091E30087FDE1CF81E01D
:1025F000E0CF81E0F5CF0F931F93CF93C82F8115C4
:1026000031F18CEF8C0F813A98F506E412E0F80175
:102610008191C81701F122E0EC34F207C9F7EFEF1E
:1026200080E0D8019D918D01C91781F0EF3F19F429
:10263000911101C0E82F8F5F863099F7EF3F31F09D
:102640000E2E000CFF0BEC5BFD4FC2839BDCCF9189
:102650001F910F910895E6E4F2E08191C81302C042
:10266000DF011E9232E0EC34F307B9F78BDCD7CFF1
:1026700080E28C0F883068F4C77081E090E001C080
:10268000880FCA95EAF7C0914204C82BC093420450
:10269000DDCF8BE58C0F833030F42C2F2452330B9D
:1026A000C901EAD8D4CFC85ACB3188F6EC2FF0E074
:1026B000EE0FFF1FE55FFD4F8081918105D9C7CFE8
:1026C000811559F19CEF980F913A60F4E6E4F2E03D
:1026D0009191891302C0DF011E9292E0EC34F90758
:1026E000B9F750CC90E2980F983050F4877091E091
:1026F00001C0990F8A95EAF7892F0E947A06F1CFD7
:102700009BE5980F933018F480E090E0B5C8885AA4
:102710008B3118F480E090E0D7C808951F93CF93D1
:10272000DF93182FEB0167DF209731F4812FC8DF8B
:10273000DF91CF911F9108958FE99FE00197F1F705
:1027400000C000002197F0CF811531F09091420434
:10275000892B8093420416CC0895811519F00E94AC
:102760007A0610CC0895811531F090914604892B9A
:102770008093460407CC0895811539F08095909197
:102780004604892380934604FDCB0895809131044B
:10279000811521F082E2F0DF109231040895A0E06B
:1027A000B0E0E5EDF3E10C94D132EC0188818115C4
:1027B00009F1813009F045C08981813051F48A8165
:1027C000239660E570E0893311F060E070E0A6DFE9
:1027D000EDCF823021F48A8123960DDFE7CF83305D
:1027E00021F48A8123966CDFE1CF843041F0229678
:1027F0008111DCCFCDB7DEB7E9E00C94ED328A81F0
:10280000239620E030E09AE0682F6053770BAB010D
:102810006A30710560F02115310551F3EFE9FFE0F1
:102820003197F1F700C0000021503109F4CF929F99
:10283000B001939F700D11249A01260F371F8991C3
:10284000E3CFE82FF0E0EC58FE4FB490282F269508
:102850002695269530E0F901EC59FE4FE4908770FB
:10286000F12C082E02C0F594E7940A94E2F7E0FAFE
:10287000EE24FF24E0F8F901EC5AFE4FC490D12C6D
:10288000082E02C0D594C7940A94E2F7C0FACC246B
:10289000DD24C0F8F901EC5BFE4F049110E002C0AA
:1028A000159507958A95E2F701701127E114F10457
:1028B00011F081EEA0DEC114D10411F086EE9BDE92
:1028C00060E070E08B2D2ADFC114D10411F086EE98
:1028D000F7DEE114F10411F081EEF2DE01151105CD
:1028E00021F060E070E08CE219DF21965FCFA1E07B
:1028F000B0E0EDE7F4E10C94C832462E1A01522EF6
:10290000C32E3701A82E880FBB08C5010E945A327A
:10291000D82E811509F46BC0C50133E0880F991FCB
:102920003A95E1F7FC01E95CFE4F2381422F50E02C
:10293000211511F041E050E0895C9E4FFC0164815B
:1029400075816F587C4FCE0101960E940934F101C8
:1029500080809180A280B38017D8681979098A098C
:102960009B09643671058105910538F4B301C801EE
:102970000E94C40B99818917D1F1E42C042C000C1E
:10298000FF08C7010E945A32D82E811106C0D12CEF
:102990008D2D2196E2E10C94E432C70123E0880FEB
:1029A000991F2A95E1F7FC01E95CFE4F2381422F34
:1029B00050E06216710408F4A301895C9E4FFC018B
:1029C000648175816F587C4F852D9C2D0E94093440
:1029D000B301C8010E94C40B99818913D8CF0E940A
:1029E000C40CF1016083718382839383D1CFA301EF
:1029F000B801852D9C2D0E940934CACFAAE0B0E011
:102A0000E4E0F5E10C94D2326B018AE0E82EF12C7F
:102A100002E713E09E012F5F3F4F4DE653E061E078
:102A200080E065DF811549F09AE0FE013196A3E66A
:102A3000B3E001900D929A95E1F79AE0E3E6F3E0B6
:102A4000D60101900D929A95E1F72A96E8E00C9450
:102A5000EE32A8E0B0E0EFE2F5E10C94D43288E089
:102A6000E82EF12C0DE713E09E012F5F3F4F4FE55D
:102A700053E063E082E03BDF182F811589F19091EC
:102A80007C0380915E03981759F100E090918003D8
:102A900080917F038917F1F0E92FF0E0EB58FC4FAC
:102AA000848587FB662760F99F5F9370909380030E
:102AB00090917E039F5F90937E038F770E94560BC9
:102AC000082F8111E3CF84E090E00E945A32102F4A
:102AD000182302C00111F7CF80917C0380935E031D
:102AE000812F2896E6E00C94F032CF92DF92EF929D
:102AF000FF921F93CF93DF9300D000D0CDB7DEB706
:102B0000C0905903D0905A03E0905B03F0905C03AF
:102B10000E94C40C6C197D098E099F0911E064366E
:102B200071058105910578F10E94D00CDC01CB0183
:102B30000296A11DB11D89839A83AB83BC838091CA
:102B40006001909161018F589C4F20915F01422F4D
:102B500050E0253010F044E050E0BE016F5F7F4F41
:102B60000E94093485E090E00E945A32182F8115A6
:102B700051F00E94C40C6093590370935A038093E0
:102B80005B0390935C03812F0F900F900F900F9039
:102B9000DF91CF911F91FF90EF90DF90CF9008953C
:102BA0008F929F92AF92BF92FF920F931F93CF93FA
:102BB000DF93CDB7DEB72B970FB6F894DEBF0FBE0D
:102BC000CDBF88E0E8E3F4E08E010F5F1F4FD8012E
:102BD00001900D928A95E1F7809135049091360429
:102BE000A091370489879A87AB87F090370480904B
:102BF000550390905603A0905703B09058030E943D
:102C0000C40C681979098A099B09E02F312F6436B1
:102C100071058105910510F4F11411F1809168019D
:102C2000909169018F589C4F20916701422F50E08D
:102C30002C3010F04BE050E06E2F732F0E940934BF
:102C400086E090E00E945A32811569F00E94C40C1F
:102C500060935503709356038093570390935803E2
:102C60001092370481E02B960FB6F894DEBF0FBEAA
:102C7000CDBFDF91CF911F910F91FF90BF90AF908B
:102C80009F908F9008950F931F93CF93DF9384307D
:102C900030F56A3020F5493010F5C42FD0E0CC0F64
:102CA000DD1F22E1629FC00DD11D112434EB839FF3
:102CB000C00DD11D1124CE0189960E942934082F00
:102CC00010E0102F0027CE018A960E942934980127
:102CD000282BC901DF91CF911F910F91089580E0BA
:102CE00090E0F8CFFF920F931F93CF93DF93F42ED2
:102CF000843070F5623060F528E0829FE001112495
:102D000034E0639FB0011124C60FD71FC750DD4FB9
:102D100081E084279E01280F311D280F311DC90134
:102D20000E942934082F10E0102F002781E090E046
:102D3000F11002C083E090E08C0F9D1F0E942934A7
:102D40009801282BC901CDB7DEB7E5E00C94F1322C
:102D500080E090E0F8CF20919C0330919D03232BDD
:102D6000C9F4703F39F4603FA9F480919A039091BF
:102D70009B0308957A3038F4693060F4843050F45D
:102D8000462F672F80CF7D3F41F4623018F441E039
:102D9000843050F080E090E008957C3FD9F76230B5
:102DA000C8F78430B8F740E09DCFA0E0B0E0EBED8D
:102DB000F6E10C94D3327C010091450480914404E7
:102DC000082BC3E0D0E010E0C8010C2E02C095959E
:102DD00087950A94E2F780FD09C02197A8F7D12CC6
:102DE0008D2DCDB7DEB7E7E00C94EF32DC2EB701C6
:102DF0008C2FB1DF0E94DC06019779F3F1CF0F939E
:102E00001F93CF93FC0187819085009789F485817A
:102E100000811181811581F0611571F0C801C5DF54
:102E2000C82F682FC8010E940006B8018C2F93DFBD
:102E3000CF911F910F910895C8010E941B06C82FC2
:102E4000F4CFCF93DF93D82FC92FAFDF6D2F7C2F17
:102E500082DF0E94DC06DF91CF910895FC0184811E
:102E60008115B1F0878190850097A1F00E94DC0662
:102E7000282F92959F709630B9F080F4925F9F70E2
:102E8000923030F4203FD1F058F481E0283E58F0E1
:102E900080E0089580819181D4DFEACF9A5FEFCFFF
:102EA00081E0243FA9F7089591E0813F09F090E087
:102EB00081E0283E08F080E0892B089581E00895A4
:102EC000382F292FCB01A32FB22F873B9105A105C6
:102ED000B10520F4875B9C4F0C94293480E0089561
:102EE00085E290E00E942934873889F486E290E0F8
:102EF0000E942934873859F487E290E00E942934EF
:102F000091E08E3F09F090E0892F8170089580E074
:102F1000FCCFA6E0B0E0EFE8F7E10C94D3320BED84
:102F200013E089E1E82E83E0F82E98E0D92E46E000
:102F300050E0B701CE0101960E941934F8018D2DA1
:102F400011928A95E9F7B8016C5F7F4F89819A8168
:102F50000E941B0BF80191838083B8016B5F7F4F48
:102F60008B819C810E941B0BF801938382838D814E
:102F700086838E818783F6E0EF0EF11C085F1F4F7A
:102F800089E4E81683E0F80691F62696E7E00C94CB
:102F9000EF32A6E0B0E0EFECF7E10C94CB32A0907A
:102FA0005203B090530381E090E0909353038093D9
:102FB00052033FE1E32E34E0F32EC12CD12C10E07C
:102FC000360100E01AC021E030E0123020F4F401B4
:102FD000859195919C01452D602F812F0E94690F4D
:102FE000539422E0820E911C39E05312ECCF0F5F14
:102FF00089E0680E711C0A3049F0C301880F991FDF
:10300000DC01A954BD4F4D01512CDDCF21E030E052
:10301000123020F4F701859195919C0141E060E028
:10302000812F0E94900F21E030E0123028F4F70148
:103030003296859195919C0140E060E0812F0E943D
:10304000900F21E030E0123028F4F701349685919A
:1030500095919C0141E061E0812F0E94900F21E059
:1030600030E0123028F4F7013696859195919C0155
:1030700040E061E0812F0E94900F1F5FB8E0EB0EEF
:10308000F11C2AE5C20ED11C143009F099CFFE01C3
:10309000319686E0DF011D928A95E9F709E113E098
:1030A0007F0146E050E0B801C7010E9468340A5F22
:1030B0001F4F0934B3E01B07A1F7B0925303A0924E
:1030C00052032696EFE00C94E732A0E0B0E0EBE686
:1030D000F8E10C94CA32FC016280448081E0848370
:1030E000EFE2F4E07490EEEAF4E0E491C0913B0486
:1030F000C695C158D0E0CC0FDD1FCD2FDD27812C28
:1031000025E0922EAA24AA94B12C55245A94E719AA
:10311000EE2EF12C80911A01881638F00E94920848
:10312000CDB7DEB7E0E10C94E632C82CD12C83E0B9
:10313000681658F4989CF0011124EE55FD4F8091CB
:103140003904808380913A04818341101CC09C9C87
:10315000F0019D9CF00D1124EE55FD4F138212825B
:10316000809118019601280F311D9C9CF0019D9CB7
:10317000F00D1124EE55FD4F4281618180810E9446
:103180006C088394C7CF9C9C80019D9C100D1124DA
:103190000E551D4FF80183818115F1F08150838315
:1031A000589EC0011124648170E00E940B33FB0122
:1031B000FF27E15DFB4F8491E82FE7195E9EC00178
:1031C0001124B7010E940B3380913B04689FB0012A
:1031D0001124F8017283C4CF0E94D833B5010E9434
:1031E0001F338C179D070CF0BBCFF3E06F1698F0E0
:1031F0000E94D833B5010E941F33F80180830E94DA
:10320000D83320913A042695622F70E00E941F3334
:10321000280FF80121839C9CF0019D9CF00D112446
:10322000EE55FD4F128280913B04893C58F088ECAA
:103230009C9CF0019D9CF00D1124EE55FD4F848364
:1032400083838ECF8431A0F784E1F2CF0F93CF93A5
:10325000DF93C8E3D4E0488159816A817B8188E0AB
:1032600090E00E945C34288139814A815B816C81C5
:103270007D818E819F8100E20E947633622F83E2FE
:1032800090E00E944A34DF91CF910F910895E8E3D6
:10329000F4E085E0808311828FEF82838383148240
:1032A000E5E3F4E082818360828388E394E0CECF1B
:1032B00080913C04833018F48F5F80933C0488E352
:1032C00094E0C4CF80913C04811519F08150809323
:1032D0003C0488E394E0BACFA0E0B0E0E2E7F9E193
:1032E0000C94D332D82F062F142FE22E30913804AD
:1032F00030FF35C0809139048D1308C090913A0495
:10330000961304C090913B04941729F090913704D0
:10331000926090933704E32FE695E695AE2FB0E0E8
:10332000A856BE4F9C91909335043C7F3430E1F415
:103330006D2F702F812F0E94E507962F672F482F42
:10334000892F0E94B0088D2F8093390400933A048E
:1033500010933B04E11419F088E394E077DFCDB7D4
:10336000DEB7E7E00C94EF32923019F410913B0491
:10337000EACF963049F3993039F3993121F7E95181
:103380008E2F8170D82EE695F0E0E15DFA4FC49162
:10339000F12C60911A01F61618F00E949208D3CF12
:1033A000FC9EC001112470E00E940B338D2FD110C0
:1033B0000CC0860F209118012F0D3327331F412F8A
:1033C000602F0E946C08F394E4CF861BF3CFE8E3F0
:1033D000F4E0818121E043816281885F7DCFE8E371
:1033E000F4E0818121E043816281885075CFE8E378
:1033F000F4E0628121E1620F08F46FEF21E0438184
:1034000081816ACFE8E3F4E0628121E1621B08F484
:1034100060E021E0438181815FCFE8E3F4E0438114
:1034200021E1420F08F44FEF21E06281818154CF06
:10343000E8E3F4E0438121E1421B08F440E021E0AD
:103440006281818149CF609138046695669570E00C
:103450004BE050E087E091E00E94EF33892B19F4B4
:1034600081E0809336040E94E80C909326038093B9
:1034700025038091370484608093370408959091E8
:10348000380490FF31C0811581F18B3280F58F7344
:10349000880F880F909138049370892B809338049B
:1034A00080913704816080933704611519F088E3B7
:1034B00094E0CCDE609138046695669570E04BE050
:1034C00050E087E091E00E94EF33892B91F00E9459
:1034D000110981E08093280320E040913B04609132
:1034E0003A0480913904F8CE089581E0D1CF8AE280
:1034F000CFCFA9DFEECF80913804869586958F5F78
:103500008B3208F081E061E0BACF80913804869573
:1035100086958A9509F48AE261E0B1CFA9E0B0E02E
:10352000E4E9FAE10C94C8328C01DC0114968C9128
:10353000811509F4BFC061E0C80161DC7C018091A4
:103540003004811136C0F8018581811509F468C005
:10355000E114F0E5FF0608F04DC0E11420E2F206A8
:1035600008F0ACC0E11437E0F30619F1F0F4C7013C
:10357000805E91090897E8F03091420480914604FA
:103580002091410499E0F801ACE1B4E001900D9282
:103590009A95E1F7F0922404E09223041092260415
:1035A000832B822B80931B0404C0E1145FE0F5069B
:1035B00019F7F8014581411183C133E7E3163CE770
:1035C000F30609F467C0A2EAEA16A2E5FA0609F4CE
:1035D0008FC208F064C2C70190528115904208F46E
:1035E00079C2B1EEEB16F10409F482C2E5EEEE16F3
:1035F000F10459C290EEE91692E5F90650F4A0E6FE
:10360000EA16A2E5FA06A8F6C7019255803491059C
:10361000B2CF970127573C472530310508F0ACCF92
:10362000F9E7EF16FCE7FF0609F04CC020912304F0
:1036300030912404232B71F1811599F081E00E94CF
:10364000030C80911B048FD889E0ECE1F4E0A2ED3B
:10365000B3E001900D928A95E1F780912604809362
:10366000D10386E0F801A2EDB3E001900D928A95B6
:10367000E1F78091D1038093300482ED93E04EDF37
:1036800010923004D80115968C91811103C080915D
:103690001B0472D8809147048770811559F0F80196
:1036A0008581811539F08091A00482FF03C082E0FA
:1036B0000E945F062996E2E10C94E432F8018681CB
:1036C000803159CFBAE7EB16BCE7FB0609F071CFA2
:1036D000811509F4CAC0A0902304B0902404E0919D
:1036E0001B04E887E983BE016F5F7F4FC5010E941D
:1036F0001B0B2C01F981F987FBEDCF2EF3E0DF2EB8
:10370000EE24E394F12C22242A94D60117963C90BF
:10371000179733FE54C06D907C90119712968D9040
:103720009C90139746145704B9F41496BC91BF8328
:10373000232DF60146816B2F89850E94350B81155B
:1037400059F08F810E946C05281634F4D601159625
:103750009C917401F92A282E48145904C9F431FEA9
:1037600017C0F601F581FF83232DD60116964C91E3
:103770006F2F89850E94350B811551F08F810E9432
:103780006C0528162CF4F60194817301F92A282E71
:1037900030FE15C0FFEF2F1212C021E0E216F10437
:1037A00071F4232DD60116964C9160E089850E9414
:1037B000350B811521F0F60185817401F82AF8E0B6
:1037C000CF0ED11C2BE134E02C153D0509F09DCF27
:1037D00031E0E316F104F1F5988592959F704885E4
:1037E000942B9F7081E0403108F480E0F82EF29431
:1037F000E0EFFE22F92AA11450E2B50620F5A1144B
:1038000081E0B80608F055C0EA2C8F2D8D704A2D46
:10381000811509F451C06AE083E09AE00E94140C1B
:10382000282F30E02115310551F44E2D66E185EE4B
:1038300099E00E94140C282F30E0811549F0F9011D
:10384000FF297F0107C0C50190528115904390F177
:10385000E12CF12C87E0E7E2F4E0DF011D928A958C
:10386000E9F7F0922F04E0922E0480912E049091BB
:103870002F04892B09F40ECFF8018581811539F0C9
:103880008FEF0E94030C809126048093250486E02C
:10389000F801A7E2B4E001900D928A95E1F78091DA
:1038A00025048093300487E294E038DE10923004DF
:1038B000F1CEFB28BB24A8CF68E08BEF99E0AECF18
:1038C000C70197578038910508F0D5C5BE2CF0E1A7
:1038D000EF1608F0DFCE66EB70E080E090E0F0DA03
:1038E0008111D8CEC12CD12C7601B11045C074E025
:1038F000272EAE014F5F5F4F5E834D83AD81BE814A
:10390000E22D1D92EA95E9F746015701FFEF8F1A64
:103910009F0AAF0ABF0AC701B601D2DA89838115AF
:1039200009F4B8CE813009F0A5C02601370122E0A4
:10393000420E511C611C711CC501B401C1DA382E44
:103940008A83811509F4A6CE8FEF830D833038F575
:10395000C301B201B5DA8B83811521F0CE01019646
:103960000E94CF134601570133E0830E911CA11C26
:10397000B11C75016401C2CF27EBC216D104E1046A
:10398000F10409F487CEC701B6019ADA3FEFC31AF2
:10399000D30AE30AF30A8111EFCFBA94A6CF8BEFD3
:1039A000830D833090F54601570143E0840E911C4E
:1039B000A11CB11CC301B20183DA8B838115C9F24A
:1039C000C501B4017DDA8C83811108C0460157011D
:1039D00054E0850E911CA11CB11CCBCFAB80BC80E8
:1039E00081E0A8168FEFB80610F0BA2CAA2496E052
:1039F000391641F0A7E03A1611F0C501A7D7C50165
:103A0000D7D7E4CFC501A2D7E1CFB4E0530142013B
:103A10003B12AFCFC301B20153DA782E46015701F2
:103A2000E4E08E0E911CA11CB11CC701B6016D5FB4
:103A30007F4F8F4F9F4F44DA711409F42BCE8115BD
:103A400009F428CE8150990B4FEF489F9001499F70
:103A5000300D1124472D4150550B240F351F215097
:103A6000310908F486CF8FE99FE00197F1F700C094
:103A70000000F5CFCE0101960E94CF137ACF1092AD
:103A800042040E9482060E948F0C88579C4E90939D
:103A900033048093320481E080933104FBCDF2EB58
:103AA000EF16F2E5FF06E9F525EE30E02770332743
:103AB00081E090E001C0880F2A95EAF72091340454
:103AC000309131043115E1F04115A9F0282B2093F4
:103AD0003404E0CDD80116968C91803110F58F2DED
:103AE00099278F7199278230910511F04297DBCF8A
:103AF00021EE30E0DBCF8095822380933404CACD61
:103B0000322F3823311569F0982F90959223909396
:103B100034040E947A06D80115968C91811509F417
:103B2000B9CD80913104811509F46DC0C090420473
:103B3000D09041040E948F0C88579C4E9093330480
:103B400080933204F8018581811509F45CC08D2DC4
:103B50008C298D79811182C0E114F0E5FF0608F50A
:103B6000E11420E4F20608F083C036EEE316F10417
:103B700009F449C0C70190528115904208F07FC0F6
:103B8000D80116968C91803108F460C0C70199273E
:103B9000109246048D32910509F582E08093460427
:103BA00072C0B0EEEB16B2E5FB0608F03FC0E0ECE9
:103BB000EE16E2E5FE0638F5F0EAEF16F2E5FF064E
:103BC000E8F420E6E21622E5F206E8F4C701925591
:103BD00080349105C0F010924604C7018E329105E1
:103BE00008F05EC08832910508F04BC08E31910517
:103BF00008F049C004974A9780F230C034EBE316CE
:103C000032E5F30641F7F8019581911509F429C4CD
:103C1000809142048272F701E052F847EB30F105DF
:103C200008F088C0E851FB4C0C94323349E7E416A5
:103C30004CE7F40630F457E7E5165CE7F50618F7AD
:103C4000CACF8BE7E8168CE7F806DCCF8F2D8F7193
:103C50008431C9F2863111F4109246040E94C613D1
:103C60008091420490913404892B80934204CBCFFD
:103C7000D80116968C91803108F088CFC4CFC70147
:103C800087CF8A9759F780913404811531F080915C
:103C9000460492E08927809346040E94C20FB3CF66
:103CA0008C34910581F38D329240ECCF80913804B1
:103CB00080FF10C08E7F8093380488E394E0C6DADA
:103CC0000E941109809137048160809337040E941B
:103CD0009208E0CC81608093380461E086958695F7
:103CE000CEDBD8CC811521F010DCD4CC8115E1F3EA
:103CF00002DCD0CC811521F072DBCCCC8115E1F354
:103D000066DBC8CC811521F07DDBC4CC8115E1F3E5
:103D10006EDBC0CC811521F08BDBBCCC8115E1F3CF
:103D20007CDBB8CC811521F0CDDAB4CC8115E1F380
:103D3000BFDAB0CCF7E7EF16FCE7FF0609F128E79A
:103D4000E2162CE7F20629F19701205E3245203277
:103D5000310520F5911122C03E2D3F7181E090E0A8
:103D6000AC0102C0440F551F3A95E2F77A01642F67
:103D700083E090E00E944A348E2D0E948C058ACC0C
:103D800081E00E94920543E062E081E00E943606F5
:103D900081CC82E0911509F46BC3F3CF40914004CC
:103DA00080914504282F30E02095309570E0242341
:103DB0003723232B19F04823409340045BE7E51693
:103DC0005CE7F50641F4911509F464CC0E946F0597
:103DD0000E94DC0B5FCC80E4E81682E5F80608F070
:103DE00096C0A0E2EA16A2E5FA0608F0BFC0E11408
:103DF000B0E5FB0608F066C0E114E0E4FE0608F05A
:103E0000CBC0D80117968D919C91009709F4FEC004
:103E10000E94DC06D82EF92ED8011596BC90159775
:103E20001696AC90A2942FE0A2228091470487704E
:103E3000811509F1CB2CB114F9F0892F807F8034E2
:103E400069F080E28D0D8830B0F0892F807E80325D
:103E500029F4B2E0DB1678F0A11469F08091A00497
:103E600082FF09C082E00E945F068091470487704C
:103E7000CC24C3948111C12C8F2D82958F708830F2
:103E800009F4E7C108F0F6C0843008F0D7C0EF2D80
:103E9000EF70EE2E823008F4FEC08F2D807F8032CE
:103EA00019F0E29480EFE822D11409F42CC131E03A
:103EB000D31609F490C1B11409F49CC1A11409F4FA
:103EC00040C100C1970130552115324008F099CF0B
:103ED000970145E0369527954A95E1F7822F8F7037
:103EE0002091400430E041E050E0082E02C0440F31
:103EF000551F0A94E2F724233523232B09F481CF9D
:103F0000911166CF109242040E94C20FC3CB970159
:103F1000205C32452032310548F1911509F471CF0A
:103F2000BAE5EB16BCE7FB0609F46CC008F04EC01E
:103F3000F1E0EF16FCE7FF0609F462C023E0E216A9
:103F40002CE7F20609F456C0E1143CE7F30609F049
:103F500058CF0E9411108FEF94E3ACE08150904055
:103F6000A040E1F700C000000E94970E8E2D8F71D7
:103F70002091400430E041E050E0082E02C0440FA0
:103F8000551F0A94E2F724233523232B09F439CF54
:103F9000911509F47FCB1CCFD80116968C918031F6
:103FA00008F02FCF91112DCF2F2D2F7081E090E0B1
:103FB00002C0880F991F2A95E2F72091400430E053
:103FC00082239323892B09F41CCF64CB4BE5E416A1
:103FD0004CE7F406C9F08091A004002482FF03940A
:103FE000802D5CE5E5165CE7F50609F00ACF0E9436
:103FF000520F07CF6FEF7FEF80E090E00E946434B4
:104000000E94231081E0F3CF80E0F1CFF801858199
:10401000C080D180811569F0C6010E94D516F82EA6
:10402000682FC6010E940006B6018F2D0E94AB16B4
:10403000EFCEC6010E941B06F82EF6CF843009F49D
:10404000EBC0C11409F437C18091470480FD33C12E
:10405000D80115961C928695869586950E949205A4
:10406000C8015CDA809147048695869586950E9402
:104070009C0521C1893009F463C18A5F8F70823049
:1040800000F7F2EFDF126FC18F2D8F71B11068C191
:104090000E9492050CC120E1F21618F0E29490EF14
:1040A000E922B114B9F0E11469F080E28D0D883095
:1040B00010F0D11009C0809142048E2980934204EF
:1040C0000E94C20F8D2D2FC0809146048E298093AF
:1040D0004604F6CF8D2D0E946013E11409F4B1CF90
:1040E00080E28D0D883010F0D11004C08E2D0E941A
:1040F0007A0606C0E094809146048E21809346049F
:104100000E94C20F9ECF8091A00482FD16C0B11400
:1041100069F0E11439F0809142048E2980934204C1
:104120000E94C20F80E00E94FB128BCF80E00E94B1
:104130006013E11409F485CFD9CFB11471F1A11046
:1041400004C08E2D0E94A4137CCF41E0A41211C0A4
:10415000F09041048E2D8F21E81609F472CF0E9451
:104160008F0C90934B0480934A04FE28F0924104F4
:1041700068CF55E0A51265CF8E2D0E94A4138E2D19
:104180000E94AF0C809143049E2D9823E91609F4F8
:1041900058CF8E298093430454CFA11012C08E2D86
:1041A0000E94AD138E2D0E94AF0C809143049E2D72
:1041B0009823911509F445CFE094E822E092430456
:1041C00040CF81E0A8123DCF809142048E2181151D
:1041D00009F437CFE4CFB11429F096E0A91608F01E
:1041E00030CFAFCFA5E0AA1608F02BCF8E2D0E94BE
:1041F000AD1327CFA114D1F3B9E3DB1209C0EFEF60
:10420000F7EE23E0E150F0402040E1F700C000006D
:104210008D2D0E94601315CF8F2D86958695837006
:10422000811569F0813009F00CCF8D2D9F2D937091
:10423000B11002C080E090E00E94640C02CF8D2D8E
:104240009F2D9370B11002C080E090E00E943C0C62
:10425000F8CE8F2D837081113BC0B11028C04D2D39
:10426000429546954770440F440F8D2D8F70042E54
:1042700001C0880F0A94EAF72D2D2071D4FE07C0E3
:104280002FE030E001C0220F4A95EAF720953F2D3C
:104290003695369533703230B1F0333091F040912D
:1042A0004404313069F0822B84230E948C050E94E3
:1042B000290C0E94820560E0C8010E94FF16FAC91D
:1042C000842B822BF2CF822B909144048927EDCF4F
:1042D000B11459F1F0FEEBCF4D2D42954695477044
:1042E000440F440F8D2D8F70042E01C0880F0A9447
:1042F000EAF72D2D2071D4FE07C02FE030E001C079
:10430000220F4A95EAF720953F2D36953695337062
:10431000323089F0333069F040914504313041F05A
:10432000822B84230E948F05C2CF8230A8F6BFCF94
:10433000842B822BF7CF822B909145048927F2CFD3
:104340003F2D3F70F32EB11439F0832F0E94920558
:104350008D2D0E94A413ABCF8D2D0E94AD138F2DF8
:104360000E949C05A4CF43EFD41680F450EFD516DD
:10437000E1F081EFD816A1F0B11409F460C0A114E6
:1043800009F45AC08D2D0E94FB1291CF93EFD916DC
:10439000F1F0A4EFDA12F0CF8091A00482FD23C0E7
:1043A0008F2D8F71B114E1F273CEB11469F0B5E0C5
:1043B000AB1608F07CCF2F2D2F7181E090E001C06B
:1043C000880F2A95EAF7B8CFE6E0AE16F2CF80E084
:1043D000B11409F4A7CF9F2D9F7181E001C0880F10
:1043E0009A95EAF79FCFB114C1F080914704877086
:1043F000843049F410924704109249041092480402
:104400008F2D8F71ADCFF5E063E0AF1608F04FCF81
:104410008F2D8F710E949B0C4ACF25E0A21640F091
:1044200010924704109249041092480464E0F0CFBF
:1044300081E00E945F063BCF8F2D8F7129CEA114A2
:10444000F9F239E3D31209C04FEF57EE83E0415040
:1044500050408040E1F700C000008D2D0E946013A5
:1044600026CFF7E7EF16FCE7FF0609F068CC81E0FE
:104470000E949C0588CC23E7E2162CE7F20609F09F
:10448000A2C880913104811509F4F9CA0E94C613AB
:1044900001C980919C04803178F480919B0481153E
:1044A00059F0E0914D0420914C04309197044091D3
:1044B000960459E02E1301C008956E2F70E05E9FA0
:1044C000F0011124DF01A25BBB4F14968C9114976D
:1044D000811559F111968C911197831326C08C91F7
:1044E000841323C015968C91159781111EC01296C6
:1044F0008D919C91A0919804B09199048A1B9B0B7B
:10450000883C910590F480919C048F708061809329
:104510009C04EC5AFB4F80818F708061808386E918
:1045200094E00E948E1A0C945506FB013196E770B8
:10453000C1CFAFE0B0E0EFE9F2E20C94CC328C01F5
:1045400086E0F801DE011A9601900D928A95E1F756
:10455000F801F580848196E9892E94E0992E609087
:104560009A04611017C0811591F0F11409F417C174
:10457000C8010E942E17811509F411C189E0F801C4
:10458000A6E9B4E001900D928A95E1F782DFFF245D
:10459000F39456C07080A280B380D0909B04209189
:1045A000980430919904A501421B530BD11409F4CE
:1045B000C6C0483C510508F079C0811541F380918F
:1045C0009704C180E0909C0450E1E51608F059C0C2
:1045D000C81215C080919604871111C0F1104BC00C
:1045E0008E2D8F70806180939C0486E994E00E94F8
:1045F0008E1A80919C04F8018683F12C21C0F11061
:104600003AC040E06C2D872D0E94520E40E06C2D88
:10461000872D0E94520EF82E8111EFCF8A859B853F
:104620000E942117292F22952F70903470F49F70CB
:104630002230A0F09115B1F0F8019681903190F4FC
:104640008F2D2F96EEE00C94E8322A5F2F702230E7
:1046500068F0C8010E948E1AFD2CF2CF911511F05E
:10466000811571F3805E883058F3F3CF803F40F3BB
:10467000815F8330F9CF80919C04816080939C049A
:10468000BCCFC8123BC080919604871137C0F1108F
:1046900035C0E682C8010E948E1A89E0F801A6E9B9
:1046A000B4E001900D928A95E1F771CFE0909C04FF
:1046B000F0E1EF1650F486E994E00E948E1A89E04A
:1046C000F40111928A95E9F798CF811509F45FCF2B
:1046D00090919704F8018181981310C080919604FD
:1046E00087110CC0F1100AC0E682C8010E948E1A20
:1046F00089E0F40111928A95E9F749CFC8010E9437
:104700002E17811509F44BC0F11409F448C08091AB
:104710009C04803208F432CF1E821F8218861986CC
:1047200080919604909197049A838983BC82AB828E
:104730006D82EF82CE0101960E948E1A1FCF483CF7
:10474000510508F0BCCF811509F421CFF11439F1DE
:10475000909197048181981318C0809196048711D5
:1047600014C080919C0480FD98CF803108F495CFCF
:104770008683807F803F09F48DCF8681982F907F3C
:10478000905F8F70892B868385CFC8010E942E177A
:104790008111F4CE80919C04816080939C04C801B7
:1047A0000E948E1AF4CEA1E2B0E0E9EDF3E20C949F
:1047B000D6324C8F5D8F6E8F7F8F88A3192F99A370
:1047C000911110924604198E1A8E1B8E86E0FE01FE
:1047D0007C96DE01539601900D928A95E1F708A12F
:1047E0008091A00482FF1FC00E948F0C209148047A
:1047F00030914904821B930B8838934138F08091A3
:10480000470482FD03C082E00E945F060E948F0C75
:1048100020914A0430914B04821B930B88389341BA
:1048200010F00E948206011561F00F8B188F61E075
:10483000CE0143960E94FF1661E0CE0143960E948E
:10484000FF160F8B188F89E0FE017396DE011A9612
:1048500001900D928A95E1F7CE010A966ADE8111E8
:1048600010C020914C0430914D0489E0FE013A962D
:10487000DE01119601900D928A95E1F78E858111E6
:104880000BC019E080914D0490914C0489132BC00A
:10489000A196E4E00C94F232822F90E001968770AA
:1048A00099273817190671F40E94111010924C04C0
:1048B00010924D0489E0E6E9F4E0DF011D928A954B
:1048C000E9F7DFCF99E0929FD0011124A25BBB4FA3
:1048D000FE01319601900D929A95E1F780934C0478
:1048E0000E945506CECF189FC0011124825B9B4FBA
:1048F00020DE811569F280914D0490E00196877069
:10490000992780934D04BECFA6E0B0E0EAE8F4E238
:104910000C94D6320E948F0C8C0180919E03909152
:104920009F038017910771F019821A820E948F0CE1
:10493000BC0149815A8180E090E035DF10939F03EC
:1049400000939E032696E4E00C94F232A6E0B0E0D9
:10495000ECEAF4E20C94D6328C0190939B038093A2
:104960009A03011580E21807B0F4C801805E91092E
:10497000089728F063EB73E10115110511F464EA5F
:1049800073E1C8010E944005802F0E94FB12269609
:10499000E4E00C94F23280EF89838A830E948F0CCA
:1049A0008160BC0149815A8181E091E0FCDEEFCF5A
:1049B000A6E0B0E0EEEDF4E20C94D6328C019093D8
:1049C0009B0380939A03011580E21807B0F4802FAF
:1049D0000E946013C801805E9109089728F06CEB73
:1049E00073E10115110511F46DEA73E1C8010E942C
:1049F00040052696E4E00C94F23280EF89838A83A6
:104A00000E948F0C8160BC0149815A8181E090E055
:104A1000CADEEFCFACE0B0E0E0E1F5E20C94D232D8
:104A200080E01CEF0DEFFF24F39490912E03209172
:104A30002D03291709F441C0E92FF0E0E15DFC4F97
:104A4000808187FBCC24C0F8D82EE894D7F89F5FEC
:104A5000937090932E0390912C039F5F90932C035F
:104A600087FD07C0DF8218870E948F0C23E0E22EAB
:104A700006C0DF8208870E948F0C32E0E32EBC0163
:104A800089879A87EB86FC864F8158858E2D91E029
:104A90008ADED982C11479F00A830E948F0CBC018E
:104AA0008B839C83ED821E8249815A818E2D90E0FA
:104AB0007ADE81E0BACF1A83F0CF2C96E8E00C942E
:104AC000EE32AFE1B0E0E7E6F5E20C94CA32FE0167
:104AD000319684E1DF011D928A95E9F766E2E62EC0
:104AE00061E0F62E8F017BE2672E71E0772E2F01B9
:104AF000AA24A394B12CF6E28F2EF1E09F2EF701A9
:104B000081917F018F3F09F444C0F894E82FE2952A
:104B1000EF70F0E021A18F70A50102C0440F551F76
:104B20008A95E2F7CA01922F982B91A392A18095C2
:104B3000892382A3789400C0EDE1F1E021E030E028
:104B4000C12CD12C41914F3F79F0A42FA295AF7089
:104B5000A05EB0E08C9190E04F7002C09595879573
:104B60004A95E2F780FF8FC080E090E0C82AD92AFA
:104B7000220F331F8E169F0629F7F70182918F3F70
:104B800011F00E94C70750EA5A95F1F7D801CD926B
:104B9000DC920E5F1F4F6E147F0409F0B0CF44E12A
:104BA00050E0B20184EF92E00E94FC339C01892B1B
:104BB00041F084E1F201A4EFB2E001900D928A95F8
:104BC000E1F70091090310E0000F111F025C1C4F78
:104BD000232B09F45AC081E0809355020E948F0C68
:104BE000909354028093530280919803811509F4A5
:104BF000A8C07E01B5E1EB0EF11C8AE0F70111922D
:104C00008A95E9F7809156028A3008F062C04EEF2B
:104C100054E1B701C8010E94180F811509F47FC043
:104C200049E255E1B701C8010E94180F811509F446
:104C300076C045E755E1B701C8010E94180F8115FC
:104C400009F46DC040ED55E1B701C8010E94180F8D
:104C5000811509F464C0109256028091080390E017
:104C6000880F991F4AE050E0B701825C9C4F0E9478
:104C7000FC3321E020935202892B09F041C06F964A
:104C8000E0E10C94E632C90171CF809155028115A3
:104C900009F4AACFE0905302F09054020E948F0CC6
:104CA0008E199F09059708F49FCF4AE050E064EF02
:104CB00072E0C8010E94FC33892B41F08AE0E4EFE6
:104CC000F2E0D80101900D928A95E1F71092550219
:104CD0008BCFC0905002D09051020E948F0C8C1943
:104CE0009D09843F914008F092CF80915202811536
:104CF00031F28AE0D7011D928A95E9F710925202AB
:104D0000A0910803B0E0AA0FBB1FA25CBC4F8AE0D1
:104D1000FE01759601900D928A95E1F7B0CF8091D2
:104D200056028F3F39F40E948F0C9093510280936A
:104D30005002DBCF8F5F809356028A3008F48DCF0C
:104D4000F2CF8AE0F801A2E7B3E001900D928A95D4
:104D5000E1F76AE070E082E793E00E94C40B809381
:104D6000710388E0EBE2F3E0ADE7B3E001900D9270
:104D70008A95E1F768E070E08DE793E00E94C40B4C
:104D800080937C03C0908503D0908603E0908703D6
:104D9000F090880380914C0290914D02A0914E02B8
:104DA000B0914F02C816D906EA06FB06B1F0C092D0
:104DB0004C02D0924D02E0924E02F0924F020E94BD
:104DC000C40CC61AD70AE80AF90AC0929403D09212
:104DD0009503E0929603F09297038BE0E9E8F3E005
:104DE000DE01559601900D928A95E1F7F0908A03C5
:104DF000E0908B03D0908C03009192031091930369
:104E000010929303111509F43ACF10FF0DC08D894C
:104E100080FF1EC09091380491609093380460E048
:104E2000869586950E943F1A11FF06C020E04D2D01
:104E30006E2D8F2D0E946C1912FF04C0011559F0C0
:104E40000E94231A13FF1BCF81E08093280317CF02
:104E50000E941809E9CF0E941109F4CFA0E1B0E047
:104E6000E4E3F7E20C94CA32FE01319680E1DF01FF
:104E70001D928A95E9F70CE010E099E4A92E93E0E1
:104E8000B92E27EB422E512C612C712C4F0173014E
:104E90006201B1E14B165104610471041CF080E120
:104EA000C82ED12CA601B501C4010E943B34AC0C24
:104EB000BD1C0D2C000CEE08FF084C185D086E0898
:104EC0007F080150104019F76096E0E10C94E6323B
:104ED0006FEF85E290E00E944A346FEF86E290E047
:104EE0000E944A346FEF87E290E00E944A3460E00B
:104EF00088E290E00E944A340E94C917AFDF67E859
:104F000085E290E00E944A3467E886E290E00E94E1
:104F10004A346EEF87E290E00C944A348F929F926D
:104F2000AF92BF92CF92DF92EF92FF920F93CF9307
:104F3000DF9388E090E00E9431344B015C01C8E3CC
:104F4000D4E068839982AA82BB821C821D821E8261
:104F50001F8283E290E00E942934282F30E040E055
:104F600050E060E070E080E090E000E20E945B339F
:104F7000282939294A295B29288339834A835B8375
:104F80006C837D838E839F83DF91CF910F91FF9000
:104F9000EF90DF90CF90BF90AF909F908F9008954B
:104FA000CDB7DEB7AA970FB6F894DEBF0FBECDBF60
:104FB00085B7806885BF85B7806885BF84B7877FE0
:104FC00084BF0FB6F894A8958091600088618093A3
:104FD0006000109260000FBE80E890E00FB6F89479
:104FE00080936100909361000FBE81E08093150172
:104FF00085EC97E090934302809342020E948917C8
:105000000E949B0D0E94F80D8091E20084608093C5
:10501000E200789480915403811599F08091E90021
:105020001091EC008F70179511271795182B10927F
:10503000E9008091E80083FD0E9438101F701093F2
:10504000E90082E084BD93E095BD9AEF97BD80931F
:105050006E00109294031092950310929603109292
:1050600097030E947017811101C032DF8091D80030
:1050700080618093D8002AE12A95F1F700C08091E1
:10508000D900182F117080FD04C00E949B0D109252
:1050900054031093980387988F988FE891E00197B5
:1050A000F1F700C000008FB187FB992790F990932A
:1050B000990390936F018038880B8195880F880F32
:1050C000880F8093160188E08093170180919803E0
:1050D00081110E947531EBE2F3E088E0DF011D925F
:1050E0008A95E9F780916F0191E0892780933503D4
:1050F00080916F019093380380916F0180916F01CF
:10510000811106C086E980931C0184E980931B010C
:1051100060E080E00E94770B61E080E00E94770B06
:10512000EFE8F1E03197F1F700C0000010E0809166
:105130003803181708F4CBC080916F01811124C087
:1051400085E0E0E7F1E0DE01919601900D928A950D
:10515000E1F785E0FE01B196A6E2B1E001900D9283
:105160008A95E1F789E0E6E7F1E0DE01119601902A
:105170000D928A95E1F789E0FE013196ADE1B1E04B
:1051800001900D928A95E1F780916F0190E0811175
:1051900001C095E09093090385E0891B8093080383
:1051A00006E211E0D8018D918D018F3F11F00E9430
:1051B000C707B1E00B321B07A9F70DE111E0F801B9
:1051C00081918F018F3F11F00E94C707F1E00632F5
:1051D0001F07A9F784E1EEE3F3E0DF01282F1D921A
:1051E0002A95E9F7E4EFF2E0DF011D928A95E9F7ED
:1051F000269A80E090E00E943634833E9E4F21F450
:105200000E94701781113EC063EE7EEF80E090E057
:105210000E94643460E082E090E00E944A3481E0C1
:105220008093440461E083E090E00E944A3460E0AF
:1052300074E184E090E00E9464340E94471948DEE3
:105240008091380481608093380461E0869586956A
:105250000E943F1A21E04FEF6FEF80E00E946C192F
:1052600061E08BE00E943F1A40E050E0BA018FE01D
:1052700090E00E945C3440E050E0BA0183E190E0AD
:105280000E945C3482E090E00E94293480930D03F8
:1052900084E090E00E9436349093A00480939F04B1
:1052A00010DCEFEFF6E721E0E150F0402040E1F7BD
:1052B00000C0000006DC80913E0380FF1AC06FEF43
:1052C0007FEF80E090E00E9464340E94970E60E0DF
:1052D000812F0E949A0B082F61E0812F0E949A0B68
:1052E000E12FF0E0EA5CFC4F880F802B80831F5F8A
:1052F0001ECF83E090E00E9429340E948C058091AB
:105300000A03811123C088E394E008DE809137040A
:1053100083608093370480913804843028F40E949D
:10532000471988E394E0FADD0E9484080E9411097D
:105330000E94B70B8091380480FF05C060E086951D
:1053400086950E943F1A81E080930A03809198031A
:10535000811101C0CDD78BE291E09093A10380939E
:10536000A0038091540310E402E1853009F491C058
:10537000A8DB1EE0812E13E0912E0EE3402E03E009
:10538000502ED201F401219131918D919D9143E0F4
:10539000E232F40709F489C028173907A1F33090E5
:1053A0009803BEE36B2EB3E07B2E10E0D301ED90AB
:1053B000FD903D01F401A190B1904F01AE14BF04E6
:1053C00059F1AE24BF2400E0CC24C394D12CC501F4
:1053D0008C219D21892BC1F03114B1F009831A83EE
:1053E0000E948F0C9C838B83F1E0FD8391E09701F9
:1053F0002C213D21232B09F490E09E8349815A8181
:105400006B817C818D81CFD90F5FCC0CDD1C093085
:10541000F1F6F401F292E2921F5F1A3039F60E941F
:10542000D00C48C080915403843031F180E00E9458
:10543000820510920B0348E150E00FB6F894A8954E
:10544000409360000FBE1093600083B7817F84603B
:1054500083BF83B7816083BF7894889583B78E7F3D
:1054600083BF0FB6F894A8958091600088618093FF
:105470006000109260000FBE24DBEEE3F3E0819148
:105480009191892B09F044C582E593E08E179F071F
:10549000B1F780915403853009F4C4CF0E941110F4
:1054A0000E94290C0E94820563CF2817390709F052
:1054B00076CF2ADA80919803811589F080913104A2
:1054C000811569F00E948F0C2091320430913304D1
:1054D000821B930B8F3F9F4710F40E94C61380914D
:1054E0003604811509F46FC080913504E0913804C9
:1054F000E695E695E81BE0932703853109F4CEC0D5
:1055000008F084C0893009F4BFC008F072C082304E
:1055100009F4A8C0863009F4AEC0E0EDEE2EE7E055
:10552000FE2E04EE17E080912803811561F01092A1
:1055300028030E94E80C9093260380932503109281
:105540002A03109229030E94E80C9C0180912503F4
:1055500090912603A901481B590B4F3F5F4798F5CF
:10556000409124034115B1F010922403409122038D
:1055700050912303241B350B2F3F3F4758F4405DC8
:105580005A48509323034093220320913704286004
:1055900020933704A0902903B0902A038E0D9F1DFD
:1055A000909326038093250385E293E0F801099503
:1055B0008091290390912A03892B29F4AB2819F0B3
:1055C000F1E0F0932403D0909803D11411F022DA83
:1055D000D82E80915D03811551F010925D0380916A
:1055E0002D0380932E0380912B0380932C03C12CD9
:1055F00099C08F3009F091CFE695F0E0E45BF94F68
:10560000E491EE2EF12C09E619E08DCF74EFE72E30
:10561000FF24F39409EE1AE0843209F484CF90F465
:1056200068E2E62EF12C07E61AE0883109F47BCF18
:10563000833209F072CFE7E4F6E0E590F59007EDEC
:1056400018E071CF853209F068CF8E2F63E0D7D78D
:10565000E92FF0E0EC5BF94FE491EE2EF12C05E63A
:1056600018E161CFF0E0EB5AF94FE491EE2EF12C06
:1056700004E219E058CFF0E0EE5AF94FE491EE2E33
:10568000F12C02E019E04FCFE695F0E0E15BF94F35
:10569000E491EE2EF12C07E319E045CFF0E0E75B53
:1056A000F94FE491EE2EF12C08EE19E03CCF61E0C9
:1056B0008C2D0E949A0BF82E60E08C2D0E949A0B84
:1056C000FF0C8F292C2D30E0D901AA5CBC4FEC9146
:1056D0009E2F9370891729F1EE0FEE0FE82BEC93B4
:1056E000809135038C0DEF70F0E0ED53FE4FA90172
:1056F0004D5C5C4F7A01B080DA019C91B90EB4E048
:1057000060E0BB1624F4EDEFBE161CF461E00E94CD
:10571000560B8B2DBB0C990B64E070E090D7D70132
:105720008C93C39480913803C81608F4C0CF80913D
:105730009803811511F06ED9D82AD1100E94D00C8F
:105740000E94290CF82E80913903F81639F0F09256
:1057500039030E94C40C8F2D0E948205809154034E
:10576000843009F0FECD83E08093E9008091E80069
:1057700082FFF7CD8091E80090E085FF05C00E9490
:105780006A0D811529F191E08091E8008B77809373
:10579000E800911509F4E5CDE0909C03F0909D039D
:1057A000E981E114F10491F1EE3F09F051C08A81E1
:1057B000833020F08550833008F04AC0EA81EE3013
:1057C00008F046C0F0E0ED50FB4CCE0101964AC710
:1057D00050E2E52EF12CFE0131966F018091E80038
:1057E00085FD0AC08091E8008B778093E8000E94D5
:1057F0006A0D811599F3C7CF8091F100D6018D9381
:105800006D01B1E0EB1AF10849F7BDCFE43148F47E
:10581000E11549F0E150E33130F4F0E0EF5FFA4C8C
:1058200021C7EE3F59F28FEF898312C01A8289E0B7
:105830008B830EC08A81823081F08330B1F0813059
:1058400091F70E94C40C24D76B837C838D839E8345
:10585000CE0101960E94BA0D84CD88E290E0F9D77E
:105860001B821C821D828E83F3CF80915203909104
:105870005303892B69F3FE01319682E593E0D2014F
:105880002C9111963C91B2E04B0E511C3283238334
:1058900032968415950599F7DBCF8A81823019F607
:1058A0006B817C818D819E81F3D688E290E0F2D776
:1058B000CFCF4C816B818A810E944316982789271C
:1058C00098279E838D83C4CF2D813E813227232745
:1058D00032274C816B818A810E94690FB9CF0E9467
:1058E000C917B6CF8A81823869F178F48038B1F06F
:1058F000813809F0ADCF60E08B810E943F1A8B8127
:10590000811115C00E941809A3CF833809F0A0CFD8
:1059100020E040913B046C818B8106C020E04B81EC
:1059200060913A04809139040E946C1991CF809162
:10593000380481608093380460E0869586950E94E3
:105940003F1A86CF8B8180933C0482CF8A81823834
:10595000E1F060F48038A1F0813809F079CF8091CE
:10596000380480FF10C08695869562CF833809F091
:105970006FCF809139048B8380913A048C8368CFF8
:1059800080913B0455CF80E053CF80913C0450CFB1
:105990000E94840888E394E00E94261959CF80E190
:1059A0008A8356CF1A8287EB43CF0C810D3108F0E2
:1059B0004FCF8A809B80982489249824A12CB12CD5
:1059C000FE0131967F010E0F1F2F111D0E151F05B1
:1059D00009F43ECF80E0F7EB8F169104A104B104E7
:1059E00020F4C401875B9C4F34D7D70114968C9365
:1059F000BFEFEB1AFB0AEFEF8E1A9E0AAE0ABE0A41
:105A0000E5CF8091520390915303892B09F420CF65
:105A10008C818D3108F01CCF882E912CA12CB12CBB
:105A2000CA80DB80DC24CD24DC24E12CF12C8E0127
:105A30000F5F1F4F412C512C3201481459046A0446
:105A40007B0408F005CFF7EBCF16D104E104F10495
:105A500038F4D80114966C91C601875B9C4F1AD715
:105A6000BFEF4B1A5B0A6B0A7B0AEFEFCE1ADE0A16
:105A7000EE0AFE0A0F5F1F4FE0CFF0D9E9CE84E0B7
:105A80008FCF8C818D3108F0E3CE882E912CA12C04
:105A9000B12CCA80DB80DC24CD24DC24E12CF12C69
:105AA000412C512C32018E010B5F1F4F48145904B9
:105AB0006A047B0408F0CCCE80E0F0EDCF16F2E073
:105AC000DF06E104F10418F4C6018996C2D6D801B4
:105AD0008D938D01BFEF4B1A5B0A6B0A7B0AEFEFC8
:105AE000CE1ADE0AEE0AFE0AE1CF2C81022F10E068
:105AF0002D3108F0ADCE8A819B8198278927982780
:105B00002C01612C712C803DF2E09F0708F0A0CEA3
:105B1000822E912CA12CB12C40ED52E060E070E07F
:105B20004419550966097709421751056105710540
:105B300008F48ECE2091520330915303232B09F0A9
:105B40003EC01C0129E2220E311C80FBEE24FF2402
:105B5000E0F880FF0BC088967CD69D818927982726
:105B6000892781159C4711F48FEF8D83D501C401DE
:105B7000840D951DA61DB71D80FF19C0680141E069
:105B8000C41AD108CE0105968C0D9D1D9AA789A730
:105B9000C101800F911F5DD6A9A5BAA59C91811561
:105BA0009C4721F48FEFE9A5FAA580838601FE01C9
:105BB0003196EE0DFF1D2FEFE016F10638F08E0145
:105BC0000F5F1F4FC12CD12C760125C09481858198
:105BD00081159C4711F42483258342E0E40EF11CD7
:105BE0003296EACF50ED451652E055066104710435
:105BF00030F4D80114966C91C20189964BD6BFEF50
:105C0000CB1ADB0AEB0AFB0AEFEF4E1A5E0A6E0AAA
:105C10007E0A0F5F1F4FC814D904EA04FB0410F377
:105C200017CE8091520390915303892B09F410CE23
:105C3000CE0101960E94BA0DFFEF21EE34E0F15043
:105C400020403040E1F700C000003FCB88E0E0E8B2
:105C5000F1E0DE01919601900D928A95E1F7FE0147
:105C600032968FE1DF011D928A95E9F786E08983FC
:105C700088E07F96DE01159601900D928A95E1F7F6
:105C8000E7CD8CE8898383E08A831B821C82E0CD88
:105C90000B811C81012E000C220B330B45E0000F01
:105CA000111F221F331F4A95D1F7B901A801405E89
:105CB0005F4F6F4F7F4F401751076207730708F41C
:105CC000C7CD0C38B3E01B072105310508F0C0CD66
:105CD0004D38E3E05E076105710520F04CE853E0C4
:105CE00060E070E0401B510BB801675A794F6ED5E8
:105CF000AFCD1B810C8140E0602F812F0E94721676
:105D00009827892798279A83898341E0602F812FDC
:105D10000E9472169827892798279C838B8398CD99
:105D20002E813F812C37310569F032272327322716
:105D300041E08D81811101C040E06C818B810E9426
:105D4000900F86CD809152039091530320E03CE761
:105D5000892B71F720E030E0EBCF4AE150E06FEFA4
:105D600070E0CE0107965ED5809152038983EA8266
:105D70001B8282E08C8387E08D8375CD81E090E08B
:105D800090939D0380939C0382E390E090933D0366
:105D900080933C030E948F0C90933B0380933A03C3
:105DA00057CDE114F10481F1C0903E03D0904C0333
:105DB00000913A0310913B030E948F0C801B910BC2
:105DC0008536910540F1C2FE26C0D7FE24C00E9450
:105DD0008F0C90933B0380933A0380913C03909106
:105DE0003D03019790933D0380933C03892B61F41D
:105DF00010929D0310929C0381E090E090935303D6
:105E000080935203E12CF12C809152038983EA8222
:105E100080913C030DCD82E390E090933D0380930D
:105E20003C03F2CF109253031092520311CD40E283
:105E300050E06FEF70E0F6D40BCD2B81273071F07E
:105E4000283049F1211104CD2FE1DC011D922A9562
:105E5000E9F788E08C8383E088A3FACC2C8166E0A4
:105E6000CE018196FC01362F11923A95E9F7283040
:105E700080F4629FB0011124675E7C4F46E050E0E1
:105E8000D8D480E0898386E0FE01B196DE011296C7
:105E9000F3CE8FEFF7CF6C8186E0FE013596DE0101
:105EA000919601900D928A95E1F789A19AA18115A9
:105EB0004CE7940741F42091520330915303232B74
:105EC00011F480E090E09AA389A38BA19CA1811595
:105ED0005CE7950741F42091520330915303232B43
:105EE00011F480E090E09CA38BA38FEF683060F406
:105EF00086E0689FB0011124675E7C4F46E050E069
:105F0000CE018196E5D480E089830E948917A0CCD8
:105F100080910C03811509F4BCCA90E199BD09BDBB
:105F200009B400FEFDCF8091D8008F7D8093D8000A
:105F30008091E00082608093E0008091E00081FD2C
:105F4000FCCF0E941110A5CA1F921FB61F921124E8
:105F50008F939F93AF93BF9380910B03811113C0D5
:105F600080916A0290916B02A0916C02B0916D02D7
:105F70004196A11DB11D80936A0290936B02A0937C
:105F80006C02B0936D02BF91AF919F918F911F9062
:105F90001FBE1F90189578941F921FB61F92112450
:105FA0008F939F93AF93BF9380916A0290916B02FE
:105FB000A0916C02B0916D020196A11DB11D80935C
:105FC0006A0290936B02A0936C02B0936D02BF9132
:105FD000AF919F918F911F901FBE1F9018951F9298
:105FE0000F920FB60F9211242F933F934F935F930D
:105FF0006F937F938F939F93AF93BF93EF93FF9391
:106000008091E10082FF09C08091E20082FF05C01B
:106010008091E1008B7F8093E1008091DA0080FF26
:1060200024C08091D80080FF20C08091DA008E7F4C
:106030008093DA008091D90080FFA9C080E189BDFA
:1060400082E189BD09B400FEFDCF81E08093540355
:1060500080915902811109C00E949B0D0E94F80D88
:106060008091E20084608093E2008091E10080FFF3
:106070001AC08091E20080FF16C08091E2008E7FFE
:106080008093E2008091E20080618093E200809141
:10609000D80080628093D80019BC85E080935403B7
:1060A00083E0809315018091E10084FF2FC08091EF
:1060B000E20084FF2BC080E189BD82E189BD09B483
:1060C00000FEFDCF8091D8008F7D8093D800809115
:1060D000E1008F7E8093E1008091E2008F7E8093CB
:1060E000E2008091E20081608093E200809158029A
:1060F000811509F452C084E08093540380915403C5
:10610000843009F052C082E0809315018091E10053
:1061100083FF2CC08091E20083FF28C08091E100C2
:10612000877F8093E10082E08093540310925802AD
:106130008091E1008E7F8093E1008091E2008E7F6C
:106140008093E2008091E20080618093E20042E06F
:1061500060E080E00E94C80D8091F000886080932C
:10616000F00081E08093150180931401FF91EF917D
:10617000BF91AF919F918F917F916F915F914F915F
:106180003F912F910F900FBE0F901F90189519BC43
:10619000109254031092590268CF8091E30087FF58
:1061A00002C083E0A9CF81E0A7CF81E0ADCF1F92ED
:1061B0000F920FB60F921124EF92FF920F931F933D
:1061C0002F933F934F935F936F937F938F939F93FF
:1061D000AF93BF93CF93EF93FF9309EE10E0F801D5
:1061E0008081C091EC008F70C795CC27C795C82BD4
:1061F000108280EFE82EF12CF7018081877F808369
:1062000078940E943810F8011082F701808188602C
:106210008083CF70F801C083FF91EF91CF91BF9140
:10622000AF919F918F917F916F915F914F913F912E
:106230002F911F910F91FF90EF900F900FBE0F9035
:106240001F9018958EE1489B02C08A95E1F7489B04
:10625000FECF0895589880E28A95F1F7589A0895EC
:10626000FC012BE02A95F1F728E090E080E031E096
:1062700040E14A95F1F7880F489B02C0816093275F
:1062800042E04A95F1F7000040E14A95F1F72A957E
:1062900079F720E12A95F1F729B132E03A95F1F743
:1062A000000040E14A95F1F7217092272081920F7A
:1062B00090830895A1E0B0E0EFE5F1E375C11982A4
:1062C0008C017C01E60EF11CBDDFCE010196C8DF1A
:1062D000F80181938F01EE15FF05B1F781E09981F7
:1062E000911180E02196E6E07BC1509A589A08957A
:1062F0005098589AE89AE9E6F0E080818C7F808394
:1063000008956150770B91E001C0990F6A95EAF703
:10631000692F90E021E0611108C0911599F0589A19
:1063200080E28A95F1F758980895362F3823311571
:1063300039F0589A922730E23A95F1F76695EBCF0B
:106340005898F9CF5898ECCFFF920F931F93CF93A3
:10635000DF93EC018C01060F111DF9907BDF68E0E3
:106360008F2DCFDFC017D107C1F7CDB7DEB7E5E07E
:1063700038C11F920F920FB60F9211240F931F93E3
:106380002F933F934F935F936F937F938F939F933D
:10639000AF93BF93EF93FF93CF93DF930F92CDB75C
:1063A000DEB719824FDFCE0101965ADF082F06951E
:1063B00006950695982F92959570202F2570920F2F
:1063C000292F237096959695920F9827977089811B
:1063D000892B811509F058C0083008F055C080E1BC
:1063E0008A95F1F7589A509A82E08A95F1F700C0A1
:1063F000589888E0089F80011124D801A95CBE4FFD
:106400001696ED91FC9117973097A9F06091D30102
:106410007091D40114962D913C911597260F371F3A
:1064200011968D919C911297680F791F13964C913C
:1064300013978C910995F801E95CFE4F6381611512
:1064400049F02091D3013091D40184819581820F4C
:10645000931F7ADFFFDE80E18A95F1F75898509814
:10646000589A80E18A95F1F7F801E95CFE4F608166
:10647000611549F02091D3013091D401818192813D
:10648000820F931F17DFDEDE0F90DF91CF91FF9118
:10649000EF91BF91AF919F918F917F916F915F919C
:1064A0004F913F912F911F910F910F900FBE0F9021
:1064B0001F9018950F931F93CF93DF938C0108972C
:1064C0000CF05EC0F894509A589885E08A95F1F7E0
:1064D0000000C02FC695C570802F8570C80F8C2F07
:1064E0008370C695C69593E0000F111F9A95E1F74A
:1064F000C80FC8018C2BEC01ADDE00C068E08C2F0A
:1065000000DF90E19A95F1F75098589A489B31C076
:1065100087E090E048992FC0F801E95CFE4F638165
:10652000611559F02091D3013091D4018481958176
:10653000820F931FBFDE811501F184DE80E28A9510
:10654000F1F75898509A90E19A95F1F7F801E95CC3
:10655000FE4F6081611549F02091D3013091D40143
:1065600081819281820F931FEFDE74DE789481E047
:1065700008C000C0CBCF019749F4509A589A78943C
:1065800080E0DF91CF911F910F91089500C0C2CF9D
:106590002F923F924F925F926F927F928F929F9233
:1065A000AF92BF92CF92DF92EF92FF920F931F9321
:1065B000CF93DF93CDB7DEB7CA1BDB0B0FB6F894D2
:1065C000DEBF0FBECDBF09942A88398848885F8412
:1065D0006E847D848C849B84AA84B984C884DF8083
:1065E000EE80FD800C811B81AA81B981CE0FD11D67
:1065F0000FB6F894DEBF0FBECDBFED010895992709
:1066000078E0880F991F961708F0961B881F7A95D7
:10661000C9F780950895AA1BBB1B51E107C0AA1FAB
:10662000BB1FA617B70710F0A61BB70B881F991F33
:106630005A95A9F780959095BC01CD01089597FBD7
:10664000072E16F4009406D077FD08D0E4DF07FC8F
:1066500005D03EF4909581959F4F08957095619572
:106660007F4F0895EE0FFF1F0590F491E02D0994E0
:10667000082E817006940694811D0694811D06944F
:10668000811D0694811D0694811D0694801D089528
:1066900069279627692778278727782708957DD146
:1066A000332312F48A1B9B0B01C077D1B7FF0895E7
:1066B000821B930B0895002E083090F0982F872F9F
:1066C000762F652F542F432F322F22270850F4CFD7
:1066D000220F331F441F551F661F771F881F991FE6
:1066E0000A95B2F7002D089597FD1094002E0830FA
:1066F00098F00850232F342F452F562F672F782FCF
:10670000892F912DF4CF1594979587957795679557
:1067100057954795379527950A95AAF71124002D87
:1067200008958F929F92AF92BF92CF92DF92EF9295
:10673000FF92CF93DF93EC01688179818A819B81FD
:10674000611571058105910521F464E279ED8BE510
:1067500097E02DE133EF41E050E0D1D049015A01FB
:106760009B01AC01A7EAB1E4E6D06B017C01ACEE81
:10677000B4EFA5019401EBD0DC01CB018C0D9D1D84
:10678000AE1DBF1DB7FF03C00197A109B0488883A4
:106790009983AA83BB839F77DF91CF91FF90EF907E
:1067A000DF90CF90BF90AF909F908F900895B9CF1A
:1067B00080E091E0B6CFA0E0B0E08093000190933C
:1067C0000101A0930201B09303010895FB01DC01D4
:1067D00002C005900D9241505040D8F70895FC0139
:1067E0004150504030F001900616D1F73197CF015B
:1067F0000895882799270895FB01DC0104C08D9135
:106800000190801921F441505040C8F7881B990B22
:106810000895FB01DC0102C001900D9241505040EF
:10682000D8F70895DC0101C06D9341505040E0F766
:106830000895DC01CB01FC01F999FECF06C0F2BD41
:10684000E1BDF89A319600B40D9241505040B8F72E
:106850000895F999FECF92BD81BDF89A992780B528
:106860000895A6E1B0E044E050E0E5CFA8E1B0E053
:1068700042E050E0E0CFDC01A40FB51F4150504092
:1068800040F0CB01840F951F2E9105D04150504010
:10689000D8F70895262FF999FECF92BD81BDF89AB9
:1068A000019700B4021639F01FBA20BD0FB6F89454
:1068B000FA9AF99A0FBE08950396272FECDFEADFC4
:1068C000252FE9DF242FE7CF0196272FE4DFE2CF42
:1068D000DC01CB0102C02D9105D041505040D8F7CA
:1068E0000895262FF999FECF1FBA92BD81BD20BD14
:1068F0000FB6F894FA9AF99A0FBE01960895052EEC
:1069000097FB16F400940FD057FD05D024D007FC58
:1069100002D046F408C050954095309521953F4FE0
:106920004F4F5F4F089590958095709561957F4F7B
:106930008F4F9F4F089531D0A59F900DB49F900D1C
:10694000A49F800D911D11240895B7FFF4CFF3DFAC
:10695000821B930B0895A1E21A2EAA1BBB1BFD01FB
:106960000DC0AA1FBB1FEE1FFF1FA217B307E4072E
:10697000F50720F0A21BB30BE40BF50B661F771F86
:10698000881F991F1A9469F7609570958095909566
:106990009B01AC01BD01CF010895A29FB001B39F3F
:1069A000C001A39F700D811D1124911DB29F700D18
:1069B000811D1124911D0895F894FFCF15113B11ED
:1069C00041113B1141119311B4114111BA12C71277
:1069D000561E721E761E7A1E7E1E821E861E8A1EFF
:1069E0008E1E921E961E262E412E482E792E902EF9
:1069F000AD2EBE2ED12E122F172F282C282C282C4E
:106A00001D2F162C1A2C4D2C592C642C6F2C722CEB
:106A1000A62CC82C132C112ECF2CD22CD52C012D0A
:086A20003D2D3F2D412D752D88
:106A28000100000001010201191A1B1C1D1E1F2074
:106A38002122000001000010001010F6F5F4F1F01A
:106A480037339293959431326734978C0CFD0EF05E
:106A58000CF10C130FF40E00000001000000000000
:106A680000000A01000000000000010B0000000007
:106A78000000080C000000000000000000E007040F
:106A8800140000000000000B1800000000000001C6
:106A9800333236349700F1F0F4F5F6956793370002
:106AA800BF597D4CDF1CBC81004422320001DE004E
:106AB800AC0006021F023F020001020202020606A3
:106AC800060909090909090F0F0F0F0F0F151515E9
:106AD80018191919191919191919192324252525E6
:106AE80025252500FF0100010000FFFF000001002F
:106AF80001FF007103E200E900EA00B500B600B743
:106B080000CD008301CC008A019201940121022367
:106B18000224022502260227022A02B300B4006FCB
:106B28000070009F01CB019F02A002E200E900EA89
:106B380000B500B600B700CD008301CC008A0192F1
:106B48000194012102230224022502260227022A97
:106B580002B300B4006F0070009F01CB019F02A038
:026B6800020029
:00000001FF
